:020000041100E9
:103000007FB50023284C294D03932800217C284AB2
:1030100001F0E1FA002812D103232800217C03AA41
:1030200001F080FA00280AD1224B039A9A4206D175
:10303000214B2248E360224B636104B070BD02263D
:10304000217CFE2228001F4B009601F03DFA00284B
:1030500001D00020F1E71C4BA2899A42F9D1217CD2
:10306000FF222800194B009601F02EFA0028F0D11B
:10307000E389174A934203D1164B17486361DCE793
:10308000164A9342E5D1164B164A1B68934206D95D
:10309000C02304222800217C9B0001F07EFA124B01
:1030A00012486361C9E7C0460862FF1F3442FF1F30
:1030B000813700005959530059598320F4BE00113B
:1030C000094200111462FF1F595900001662FF1FC8
:1030D00083050000BD410011D4BE0011821500001F
:1030E0002C62FF1F87130000C5420011E4BE0011CF
:1030F000002370B51A4E1B4C30006361637401F0FD
:1031000091F9402323744B2B0CD9CC233821AC22CA
:1031100030009B01217401F040FA00280AD00025FC
:1031200025740CE0FFF76CFF051E08D1237C0433E7
:10313000DBB2E7E70C4B0D4D63610D4BE381236878
:10314000002B08D1002D06D00C222900200008F009
:1031500043FE2B7B6374300001F0A2F970BDC046C2
:103160003442FF1F0862FF1F5D420011C4BE001100
:10317000AAAAFFFFF7B5164B0192C318021D002043
:10318000009388235B05D3181B685C1C1AD09CB283
:10319000402C18D88D781E0CAC466746CD782D0291
:1031A0003D43AE4206D1019800280ED110000C70AC
:1031B000240A4C7003249BB20733A343D218009B0C
:1031C0009A42DED3FEBD4432F9E71000FAE7C0466A
:1031D000FC0F0000802213B503000324019189B283
:1031E000520107319B18A14304305A1A88235B050A
:1031F000C3181B68591C03D190429241104016BD60
:1032000099B2402907D80B000733A343C018904256
:10321000ECD30020F3E74430F9E7134B134A1B6863
:10322000126810B5FA24934201D81A00F824104B02
:10323000E4021B689A4210D813000E4A12689A42A0
:103240000ED3013307D1F823DB029C4203D10A4994
:10325000054808F099FD200010BDFC24E402ECE7CD
:10326000FE24E402F7E7C04600C0071100D00711B2
:1032700000E0071100F00711FFFFFF7FF0B59BB0E2
:10328000150004900391402A00D9A0E006AB5980B4
:103290001A80FFF7C2FF0400042816D9002206A9ED
:1032A000FFF768FF052810D906AB1B88AB420CD18D
:1032B000002D07D0514B2A000499C01808F09CFA41
:1032C000002802D101201BB0F0BD06AB1D802000FC
:1032D0000699FFF77FFF041E7BD1069B0793FFF73C
:1032E0009CFF80235B01C618802307001B039E42BE
:1032F00001D3F826F60288235B05F31801931B68B7
:10330000013302D0019808F0FFFA3D49019808F016
:103310003BFD3B1D0293331D05938822029B520502
:103320009B181B6808935A1C3CD044219AB2009108
:10333000402A04D80320D11D814389B2009103990A
:103340001B0C8B4224D0402A22D80122300008A92D
:10335000FFF710FF021E1BD1380008A9FFF70AFF74
:103360000400042831D9009A059B9B188022520141
:10337000B218934240D288235B05C118009A09A86D
:1033800008F02AFD1D4B009A09A9F01808F044FB2B
:10339000009A029B9446634402931A4B029AFB18CC
:1033A0009A42BAD388235B05FC1821680198013939
:1033B00008F0EAFC200008F0A7FA039A07AB5A804D
:1033C00030000799FFF706FF0400002C03D100200E
:1033D00079E70428FBD988235B05E018069908F0F3
:1033E000D3FC0323EA1C9A4300D16BE7034B0499F7
:1033F000E01808F011FB65E70424ECE70400001175
:10340000FFFFFF7FF80F0000F7B505001400402A0A
:1034100021D8002701AE71803780FFF7FEFE042817
:1034200016D93A003100FFF7A5FE042810D93688D6
:10343000BC420BD0BD4209D0221CB44200D9321C80
:10344000064B92B2C118280008F0C6FC30B2FEBD8F
:10345000C04300B2FBE703204042F8E7040000113C
:1034600037B5042204000D0001A81649FFF7CCFF70
:10347000020004280BD1019BA34208D3AB4204D025
:10348000104901A80195FFF7F9FE01203EBD0E4C41
:1034900023682000019308F037FA019920000139D0
:1034A000019108F071FC80235B01E418074B9C42FA
:1034B000EED10422034901A80195FFF7DFFE0020A9
:1034C000E4E7C0465555000000C007110000081190
:1034D00030B589B008F0D8FB10226946254808F0BD
:1034E000C3FA254B009A9A420ED1019B029A0F2BE8
:1034F00033D8002101240698013B08D2002900D0CE
:103500000292029B013331D10023029325E0551C26
:10351000F2D102002100EFE710341022200004A9AC
:1035200008F0A2FA029B013301D1069B0293882383
:1035300004995B05C918059B06981A03120B0491A0
:103540000592814203D02B4201D108F045FC019B3A
:10355000013B0193019B002BDED1029B002B03D08A
:10356000049304984168084709B030BDE025014C38
:103570002D03EFE700000111504859368022F8B5BD
:10358000964C974BD200002120001C6008F0ACF94B
:103590002300944A88331A60934B1A786A23002ACE
:1035A00000D01133E3620A232365904B37221B7846
:1035B0000820A3638E4B2118E361102323628D4BF7
:1035C0003B256361C823DB00A36123008C331A60B1
:1035D0002823013AE26320646364CA67043A211D28
:1035E000CA672100BC310D602100C0310860210094
:1035F000C4310B6021000635CC310D602100083D3F
:10360000C8310D602100D0310A602200D432106030
:103610002200D832136022000227E0322100176016
:103620004222DC310A6021001B3DE4310D602100A3
:10363000E83108602100EC310B6023000521F433F0
:1036400019602300F0331A602300183290331A6097
:1036500023009433186023001E3A98331A60AF2376
:10366000DB002360644BFA262363644B644DE36004
:10367000644BF031A3642300FF31FC33B600A1603A
:1036800021611E60A5627325E5656D3D6565A565D3
:1036900096255D4AAD00E264666258606766A5667D
:1036A00000270925A767E566584F594D6067200038
:1036B0002567E2673A6015279C30676007001A208B
:1036C00038602000A0300700212038602000A8309A
:1036D00007004C4838602000F83006602600642758
:1036E000A436376026005F3FAC3637602600033FC4
:1036F000B03637602600C637B4363760260000275C
:10370000B836376038269E60424E96205E64424E40
:103710005A66DE61414E9A645E62F53EFF3E9E62ED
:103720001E269A67354A8000DE661F675F67DD6583
:103730001D661862DA67BE23394A5B00E250394BD6
:10374000D838235004302250C4225200A350C6233C
:10375000E4205B00E1500433334AE1503349344BF9
:10376000D1603449800019503349E938FF38195085
:1037700032490430195032493248D161324911631B
:10378000324951631900F4310860CE2030494000BD
:1037900011603049195019002F48F83108602F493D
:1037A000D16582212E4A89005A501A002D490832CB
:1037B000D1671A002C49B432116088212B4A890044
:1037C0005A501A002A49883211602A4ADA6408F0ED
:1037D0000BF8012008F0D0FAF8BDC0460004FF1F26
:1037E000A464FF1F706FFF1F7844FF1F4A0AFF1F6A
:1037F0003A07000080C3C9019A020000DC050000FE
:103800006A18000050C3000088130000F009FF1F71
:10381000204E00006509FF1F68100000C409000069
:1038200040420F0010270000FC00FF1FB11CFF1FCB
:103830000000FF1F052DFF1F8D30FF1F252FFF1FCD
:103840007120FF1F6127FF1F8D20FF1F3922FF1FDF
:10385000FD1FFF1F8529FF1F6D2AFF1F8D19FF1FE9
:103860009128FF1FB525FF1FC125FF1FFD1EFF1F4C
:10387000B51FFF1F751EFF1F0223F0B50124624D07
:10388000624E2B70624B91B01C70624F0393336891
:1038900000210820FB7006F073FE082006F06AFD88
:1038A0000023984205D0FA78552A02D0332A00D056
:1038B0009DE03360042006F0DDFF08F03DFAFFF7DD
:1038C0005DFE07F0F1FF1F2201240021524B10AED4
:1038D0001A70524B1C70524B1970524B196891431D
:1038E000163A0A431A60602219689143403A0A4323
:1038F0001A6008F069F908F0E7F84B4B9847C120C7
:10390000FF214A4B80001A588A431A50C522920060
:1039100098588843BF390143995098584449084002
:103920008021C9010143802099509958C00509029E
:10393000090A0143995080213E48490108F08CF959
:10394000032322003C49019400933C4808F014F8FA
:103950002C223B4905A808F03FFA05AC6178207895
:10396000023406F027FDA642F8D1364C0020012192
:1039700006F034FE2268344B03201A40A023DB02F9
:1039800013432360802322689B041343236022682F
:103990002E4B1A4080239B03134323602C4A2D4B4C
:1039A000934200D8012007F0DFFF07F0E5FE8023F7
:1039B0002268DB0413432360287808F0B5F8039BE2
:1039C0001878C0B208F098F807F0F6FF22490420F2
:1039D00007F0DAFE06F01AFF00F040F800F030FEC3
:1039E00000F0D8FE00F018FA002011B0F0BD0093EE
:1039F0002100194A042008F0AFF88023DB059C62FF
:103A0000FFF766FD56E7C0464A0AFF1F34F0004044
:103A10007844FF1F3862FF1F480AFF1F490AFF1F33
:103A2000680AFF1FBCF00040E1A2000000E100E0D6
:103A3000FF00FFFF7C44FF1F0057FF1F7C54FF1F48
:103A4000E8BD001114F00040FF7FF8FFFFFF9FFF6B
:103A50000080FF1F706FFF1F3B000108002210B5A0
:103A60001100112007F0D0FE10BD0000F8B50023B2
:103A70000926374F374C3B62E3681120B343E360BC
:103A800007F00AFF112008F03FF9112007F084FE2B
:103A90004023226880251343236080236268DB0271
:103AA00013436360A3682C4A2B43A360A3680221DD
:103AB0001340A3608023A2689B0113431022A360DC
:103AC000236C072093432364236C0F3A134323642E
:103AD00080235B003B62226B204B1A402263626BA7
:103AE0001A406263A26B1A40A263E26B1340E36365
:103AF000E3681B4A1340E36006F05CFC01210720E9
:103B000006F06CFD174B11205A6C15435D6408F0EC
:103B100033F8FD21144B154A89005A508023C720E1
:103B2000626B5B0313436363E36880003343E360CA
:103B30000F4B104A19581140802212020A431A50A2
:103B4000802292051A6008220B4B5A63F8BDC046CA
:103B500000F000403CF00040FFFFDFFFEFFFEFFF11
:103B6000FFFF7FFF003800400000FF1F5118FF1FBC
:103B700000E100E0FF00FFFF00000540E12010B57C
:103B8000C00407F0D9FE10BD70B52B4C238C002B60
:103B90002AD0FA22D200934201D2FFF7EFFF228A05
:103BA000238C002A21D1DA0023826382A382E3825C
:103BB00023836383A383E38322606260A260E26065
:103BC0001E4D1F4A6420EB8093420AD8FA2200203F
:103BD000D200934205D91B4A0A21981807F034FEF7
:103BE000C0B200232872238470BD0720E11CCA7F65
:103BF00001320240CA7705D10325201DC17F013162
:103C00002940C17708325200A352002321001A0034
:103C1000088A01321B180231082AF9D1221DD27FED
:103C20009200A350626823689B18A2689B18E26800
:103C30009B185B099BB2C3E77861FF1F2062FF1FDF
:103C4000B70B000030F8FFFF30B503A804880B2045
:103C5000002C0ED14968074D0878497809020143C4
:103C60000A20A94205D1012120001980024B1B7AAC
:103C7000137030BD192A00002062FF1FF7B5150030
:103C800008AA16884A680F4F147852781202224305
:103C90000A24BA4214D10122DBB2019200962A0012
:103CA00007F004FD041E0BD1074B1B68002B07D047
:103CB00068782A7800021043424250410130984708
:103CC0002000FEBD02290000A461FF1F30B50125C0
:103CD00003790400BFB02B4211D00A49408807F095
:103CE00051F828420BD0084B01A95B8D4D800B8009
:103CF000064B00221B7A60880B7104F023F93FB059
:103D000030BDC0469C61FF1FA840FF1F2062FF1FFF
:103D100010B50549054806F0EBFF0421044A0548A3
:103D200006F0A8FF10BDC0469C61FF1FFFFF00000A
:103D300014BE0011A840FF1F10B5024804F084FF14
:103D400010BDC046CD3C0011012303700B4B1A7A05
:103D50004270022282709A78C270DA78027103226D
:103D600042711A7982715A79C2710C2202729A795F
:103D70004272DB7983720B207047C0462062FF1FBE
:103D8000022310B50370013B437005338370103379
:103D90000371443B43712A3383714433C37100235D
:103DA0000372064B04001B8843720A30FFF7CCFFF6
:103DB000831D0A30C0B2E37010BDC0462062FF1FF1
:103DC00010B5142007F0F8FE124B142200211860E1
:103DD00007F08AFD002007F007FF012007F0B4FF7D
:103DE000022007F081FE032004F0D2F9042006F03F
:103DF000E7F9052003F010FC062004F0DDF80720A9
:103E000001F0B4FA082006F015FF092001F080F84F
:103E100010BDC046A861FF1F07F04EFE012007F04D
:103E20009BFF07F019FE0000094B10B504009842F3
:103E300005D0012904D12000064906F059FF10BD24
:103E40000229FCD1013904F0BDFE0028F3D0F6E7C9
:103E5000FEFF0000CE61FF1F70B50D7A100004AAAE
:103E60002C00168810221440154220D1002E20D19B
:103E70000A78022A18D14A68517815780E4A090240
:103E80002943914205D00D4A914209D01C800A2451
:103E900004E014220A491A8007F09EFF200070BD3A
:103EA0000C2208491A80F7E71C800124F6E7082451
:103EB000F4E70B24F2E7C046F3FF0000F4FF000034
:103EC0000443FF1F10BF001110B504000749084844
:103ED00006F00EFF074804F0F7FD0020E40704D5C4
:103EE0000721054A054806F0C5FE10BDCE61FF1F3B
:103EF000FFFF0000293E001158BE0011EC40FF1FDB
:103F000000B50C4BBFB01A780B4902A800F0FCFCBE
:103F10006B4680B2D880002809D06A46074B01A9B9
:103F20001B889380064B0022188804F00BF83FB0E2
:103F300000BDC046AC61FF1FAD61FF1F4641FF1FC2
:103F40005042FF1F00B50C4BBFB01A780B4902A8B6
:103F500001F03EFF6B4680B2D880002809D06A4647
:103F6000074B01A95B8D9380064B0022188803F054
:103F7000E9FF3FB000BDC046D661FF1FD761FF1FFC
:103F8000EC40FF1F5042FF1FF7B50E00377A1C00B0
:103F900008AB11003D001A8820231D401F423CD170
:103FA0003378022B3BD173681F785B781B023B434D
:103FB0001E4FBB4208D01E4FBB4214D01D4DAB421A
:103FC00021D00A252800FEBD002A2AD1142C2AD887
:103FD0002200F06807F000FF174B1C70012CF1D98C
:103FE000FFF7B0FFEEE7002A1BD1202C1BD82200E0
:103FF000F06807F0F1FE114B04211C70104B18788B
:1040000007F082FDDEE7E3B20124009201940A008A
:10401000310007F04BFB0500D4E70825D2E7012566
:10402000D0E70B25CEE70D25CCE7C046F3FF000017
:10403000F4FF000002290000D661FF1FAC61FF1FE2
:104040005862FF1F332310B5040003700A2207498A
:10405000013007F0C1FE064B0F201B681A0AE372FD
:1040600022731A0C1B0E6273A37310BD2062FF1F14
:104070004862FF1F30B5012503790400BFB02B4211
:1040800013D00B49408806F07DFE28420DD06A46C9
:10409000084B02A81B889380FFF7D4FF6B46D8809B
:1040A0000022608801A903F04DFF3FB030BDC0463B
:1040B000CE61FF1F4641FF1F10B5024804F0C4FD4A
:1040C00010BDC0467540001170B5160004AA1488D2
:1040D00005AA15784A685078117800022A4A0843E0
:1040E000801805284BD807F0BFFD03131E29343F65
:1040F0000720042C0BD80522121BAA4200D92A0043
:1041000022491A803000091907F066FE002070BDB0
:104110000720112CFBD81222121BAA4200D92A0018
:104120001B491A80EEE707200E2CF0D80F22121B35
:10413000AA4200D92A0017491A80E3E70720032C76
:10414000E5D80422121BAA4200D92A0012491A807B
:10415000D8E70720032CDAD80422121BAA4200D980
:104160002A000E491A80CDE70720032CCFD804225D
:10417000121BAA4200D92A0009491A80C2E700226C
:104180000A201A80C3E7C046DCD5FFFFA3BE00119A
:10419000F461FF1F93BE00118EBE001189BE001195
:1041A00084BE001110B50D21024A034806F062FDDD
:1041B00010BDC04678BE00115C41FF1F13B5104C06
:1041C0000423217C01AA00F0ADF9002815D16B462B
:1041D0009A88236852BA92B25343228909491B0C28
:1041E0009B184B806B46DA88636852BA92B253438D
:1041F00062891B0C9B188B8016BD0120FCE7C04612
:104200000862FF1F2062FF1F13B5124C06236A4687
:10421000217C00F087F9002819D16B4619882368A2
:1042200049BA89B24B4321890B4A1B0C5B18538056
:104230006B46D97803335B781B020B435BBA61682A
:104240009BB24B4361891B0C5B18938016BD012008
:10425000FCE7C0460862FF1F2062FF1F37B5174CFE
:1042600007236A46217C00F05DF9002824D16B46C3
:104270001B787F2B20D86B46DD78F0232A041B03A4
:104280001A406B469B880E495BBA9BB21A4323685F
:104290002D09534322891B0C9B184B806B465A787F
:1042A0009B7812031B011A4363682A4353436289B4
:1042B0001B0C9B188B803EBD0120FCE70862FF1F92
:1042C0002062FF1F7FB50226154C0022217C03AB24
:1042D0000096050000F0F8F8002802D0012004B094
:1042E00070BD0E23217C0122280000966B4400F053
:1042F000EBF80028F2D16B469A892368D2BA53436F
:10430000228908491B149B184B806B46DA89636825
:1043100052BA92B2534362891B0C9B188B80DEE722
:104320000862FF1F2062FF1F70B5184C237C002B12
:104330000FD0382B0ED1164D280000F073F8CC2387
:10434000AC222800217C9B0100F027F9280000F016
:10435000A7F870BDE3890F4A934209D10C4D28009C
:1043600000F060F800222800217C00F005F9EDE75C
:10437000094A9342EDD1064D280000F053F89022EF
:104380002800217C920100F026F9DFE70862FF1F78
:104390003442FF1F830500008320000070B5144CD9
:1043A000237C002B1FD06369002B1CD0114D2800EB
:1043B00000F038F86369280098470400280000F0EE
:1043C0006FF8002C10D10C4B0422995E002905DAFD
:1043D0009C801A8801321A80200070BD074A9142E1
:1043E000F7DD9A80F5E70124FEF782FEF4E7C04688
:1043F0000862FF1F3442FF1F2062FF1F0F270000CB
:1044000010B58024064AA4001168436B234205D1ED
:1044100013685B1A032BF8D9012010BD0020FCE7BC
:104420006008FF1F70B5C17905000C00631E9C4138
:104430001A4BE402E41849000460C9B2007906F09E
:1044400003F9E979687949000131C9B206F0FCF84D
:10445000E8790930C0B207F09FF90023E3666133C1
:104460002360AA795B3B002A0ED022689A43023B64
:10447000134323600A23E36107332362002323638A
:10448000A3630133E36370BD22689A43022313439D
:104490002360462363610633A361EFE700500040C9
:1044A00070B5002504000368DD66C0790930C0B22C
:1044B00007F0F2F92900207906F062F82900607906
:1044C00006F05EF870BD0000F8B51E0006AB1D7862
:1044D000002304681700E366616007F0D5FB012341
:1044E0008022E3662B0027615200013B08D207F0CF
:1044F000E3F908200A4A1168002D03D12800F8BD0D
:104500002261F2E7236F034203D02369013D337038
:10451000013613685B1A032BEED90125EEE7C0467E
:104520006008FF1F70B51C00002305681600EB66CD
:10453000696007F0A9FB01238022EB66230052008B
:10454000013B08D207F0B8F908200A4A1168002C8C
:1045500003D1200070BD2A61F2E72B6F034203D024
:104560002B69013C3370013613685B1A032BEED9BB
:104570000124EEE76008FF1F002370B504681500F2
:10458000E366616007F080FB0123E366256107F0C5
:1045900093F92000FFF734FF70BD70B51D000023B4
:1045A00004681600E366616007F06EFB0123E366B2
:1045B00026610F33626B1A42FCD02B0A2361102351
:1045C000626B1A42FCD0EDB2256107F075F920004C
:1045D000FFF716FF70BD002370B504681500E36691
:1045E000616007F051FB0123E3662B0A236110236E
:1045F000626B1A42FCD0EDB2256107F05DF9200034
:10460000FFF7FEFE70BD70B51E00002305681400A4
:10461000EB66696007F038FB0123A619EB660F33E0
:10462000B44205D107F048F92800FFF7E9FE70BD54
:1046300021782961696B1942FCD00134F0E7000050
:1046400010B5084CE368002B08D18022064B5202BB
:104650001B689B186360054B1B68236007F0D4FA46
:10466000A06010BD4862FF1FC8F00040CCF00040C1
:1046700070B5184A936A916A9942FBD116498A68C3
:104680009A421FD39A1A8B60144B0126186893B272
:10469000D202D20E4343424300204C681B0A1B192E
:1046A00012029B180E4C0A684B60551CA3420CD892
:1046B000002801D04B600A600A4A136008680A4B60
:1046C000186070BD581E821ADDE7084A30009B183A
:1046D0002A00EAE700F000404862FF1F140AFF1FAB
:1046E00040420F00C8F00040CCF00040C0BDF0FFD9
:1046F00070B51F4C23793F2B01D93F2323711D4BEC
:1047000022791A701878C0B207F0B6FA18231A493D
:104710001A4A0B801A4913800B805380A3791949D8
:1047200080200B800C21938001334B43164D191CC4
:104730000001834200D9011C2980D1806379002BBC
:1047400001D101336371237A012B01D80223237233
:104750006279237A0D4853430A21584307F074F8CD
:104760000B4D2860E379052B01D81023E37170BD50
:104770003C62FF1F480AFF1F4E42FF1F2444FF1FD9
:104780004C42FF1F4A42FF1F4842FF1F71020000B8
:104790002C62FF1FF8B520210020FEF761FE114CAE
:1047A000011E114D09D10C22104BC1CBC1C42800F0
:1047B00007F09AF8FFF79CFFF8BD0C2220000C4987
:1047C000FEF722FE0C2802D0084B43CB43C40C2238
:1047D00028000849FEF718FE0C28EBD00C22002117
:1047E000E5E7C0463C62FF1F0862FF1F04BF0011DF
:1047F000FC0C0000F50C0000F0B51D4C8022A54417
:104800000400882069465201400507F03DF99022D6
:1048100012016A441300200032C832C316C816C3FE
:104820008023144C144FA6689B033343A3603B6062
:1048300006F0BAFF8823A0685B05C01807F064F88B
:104840000025882329008022A0685B05C018401934
:104850006944520007F0E0F880230135FF355B0121
:104860009D42EED1A6603E60044B9D44F0BDC04623
:10487000FCEFFFFF9443FF1F9808FF1F0410000088
:10488000F0B5040087B0002825D0684607F0F4F89A
:104890001B4C022806D106226946200006F0ACFF18
:1048A000002816D06946002301250F262F00E25C60
:1048B000013310091030874038002F0032409740F4
:1048C0003A0002434A610439062BEFD16846FFF7EC
:1048D00093FF07B0F0BD182269460A4807F0D4F8E4
:1048E0006A46A300D358013305D01822FF21684639
:1048F00006F0FAFFEAE70134062CF1D1E9E7C046F9
:104900006509FF1F00090011F0B5002504000E0025
:1049100085B0AA4200D186E04B1C087801934B7801
:104920008978377909021943F3783F061B040B4352
:104930001F43039720706570252800D196E033D877
:10494000112813D807F040FA69002F012F012F0119
:104950002F01AA00B800B1002F012F012F012F0154
:104960002F012F012F012F010F012901232800D131
:10497000E8E0DB2800D038E1042A00D8B1E01025B7
:10498000052A05D0551F2A003800711D07F024FAAA
:1049900005223100200007F01FFA2A003900601DAF
:1049A00007F01AFA05353EE0562859D010D83328BA
:1049B00000D1A7E0552839D02628DAD1A14B29000B
:1049C000132218001D0006F08FFFFEF791FB5CE03C
:1049D000712800D177E0722800D189E0602800D1E9
:1049E00095E0DC28C5D1022A00D87AE07378BFB2FE
:1049F0006370B378A370032A05D0033A390092B2EA
:104A0000F01CFEF73BFC10223900E01CFEF7FCFC1A
:104A1000C51C002807DA607070E00C2220008A496B
:104A200007F0DAF90C25280005B0F0BD013A874DF2
:104A30000C2A13D8002A0AD02800019907F0CCF9D3
:104A4000FFF756FE0C2228008149FEF717FC2900CB
:104A50000C22601C07F0C0F90D25E4E70C22EBE7FF
:104A60007A4D7C4B2A0043CB43C2E9E7013A754DAE
:104A70000C2A11D8002A08D00199280007F0ACF9B7
:104A80000C2228007449FEF7F9FB29001322601C50
:104A900007F0A2F91425C6E70C22EDE706226F49BC
:104AA000601C07F099F90625BDE712226C49601CCD
:104AB00007F092F91325B6E708226A49601C07F04F
:104AC0008BF90925AFE7012A0ED07178F02908D8B3
:104AD000654D288801F0D8FD644B2A885200D35ACE
:104AE00000E0FF23637009E05F4A604B1288F5E73E
:104AF0005F4B012A04D072789A706270022592E7A7
:104B00009B78EFE72000FFF79DFA05008BE7013A5D
:104B1000574B584D062A10D8002A10D001212800E2
:104B20005970019907F058F901F064F8290006223C
:104B3000601C07F051F9072575E70622EEE7002211
:104B40005A70F3E7042A04D94B4D2F6007F05CF844
:104B5000A860FFF78DFD0422039003A9601C07F0F5
:104B60003BF905255FE7454D062ADFD906222800D7
:104B7000019906F041FE0028D8D0062201992800AC
:104B800007F02AF906223E492800FEF777FB0123A9
:104B9000374A91780B439370C8E7012AA1D0707807
:104BA000FFF76EFEAAE7012800D0E2E6931E354F1C
:104BB000132B06D87378002B0BD100F017F900F0F7
:104BC0004DF9314B39001D78601C6A1E07F004F95D
:104BD00029E7551E2A000199380007F0FDF8380032
:104BE0002A49AAB2FEF74AFBE9E7DA281DD1042ACE
:104BF00000D876E7082A15D9B37972791B021343D6
:104C0000F27912041A43337A1B0613433B603B6864
:104C1000052231002000039307F0DEF80422601D16
:104C200003A94CE7FE236370F1E7DE2800D058E7C4
:104C3000511E012A01D10025F5E6019800F0C0FFC0
:104C4000F9E7C0460862FF1F10BF00113C62FF1F5A
:104C5000FC0C000004BF0011F50C00001462FF1FE3
:104C6000F461FF1F9843FF1F5042FF1FA864FF1FFE
:104C70003862FF1FF442FF1F4862FF1F6509FF1FD4
:104C8000ADAC00003964FF1F3764FF1FAEDE0000CB
:104C900070477047020010B5094B0A32094C92B2B6
:104CA000DA815A8298811882207802F053FB04221C
:104CB000054B012120781A7006F026FF10BDC04672
:104CC0002243FF1F8264FF1F8164FF1F013870B5FC
:104CD000042809D806F0C8FF030928081200234B4E
:104CE0000221187806F010FF70BD204B08211878BB
:104CF00006F09AFE00221E4B1A72F5E7802200246D
:104D00001B4B1A4D52001A8108211A682878DC7250
:104D100006F03AFE2100287806F0EEFD012000F0B2
:104D200087FE00F067FFDFE7104B0821187806F0D8
:104D30007BFE1048FFF724F80F4B104A9B790020A8
:104D400093800F4A13808022094B5200D8721A8137
:104D500000F06EFE00F04EFF0A4B9B78002BC3D094
:104D6000094A136006F068FEBEE7C0465862FF1F9E
:104D70002C62FF1F5942FF1F3C62FF1F2444FF1F8C
:104D80004A42FF1F3862FF1F34F0004010B500296F
:104D90000BD1082809D1054B1B78002B05D0262202
:104DA000034B04485A72FFF775FF10BD5A64FF1F8A
:104DB0002C62FF1FC40900000300F0B50A4D8E18D5
:104DC000B14202D152008018F0BD0C782F6824093E
:104DD0003C5D0F271C700C7801313C402F683C5D16
:104DE0005C700233ECE7C0464442FF1F0E22124BB8
:104DF00010B51A700D23114C11492370093A043B68
:104E00001048637006F0E8FF2D2301220E490F4879
:104E1000E371FFF7D1FF01220D49FFF7CDFF01221A
:104E20000C49FFF7C9FF030000200B49020018706E
:104E3000FEF724FA10BDC0465664FF1F3764FF1FFB
:104E4000A3BE00113964FF1F6709FF1F3F64FF1FE6
:104E50006609FF1F6509FF1FAEDE000070B5134C29
:104E6000142220001249FEF7CFFA431E114D132BD6
:104E700019D8AB78002B16D0431C2B7009236B700C
:104E800000230019037028780B4B01302900C0B2B1
:104E9000187006F0F9FC297822000139C9B2002007
:104EA00005F006FE70BDFFF7A1FFECE73964FF1FB8
:104EB000AEDE00003764FF1F5664FF1F10B5114BB4
:104EC0001A781870002A0ED000280BD10E4B1A78D1
:104ED000062A07D85423D340DB0703D50B4B187899
:104EE00002F038FA10BD0028FCD0074B1B78012BCC
:104EF00002D0033B022BF5D8044B0121187806F0B1
:104F000003FEEFE75A64FF1F8164FF1F8264FF1FE7
:104F100070B5514E514A52493070082005F054FC8A
:104F20000121022005F05AFB022005F03BFC012183
:104F3000002005F053FB002005F034FC00F0E4FEF7
:104F4000FEF7D6F806F0C8FC032246494648FFF7AC
:104F500033FF2D24030004221C7044490130FFF765
:104F60002BFF30230470424D424C437083702E3B24
:104F7000062220004049EB87FEF746FA062813D0A8
:104F8000200006F079FD022809D00321200006F058
:104F900023FD8D23E3706E3B237119336371062269
:104FA00020003549FEF76AF9344B1B68FC335C641A
:104FB000FFF754FF0020FFF781FF314C314A0121F8
:104FC000314B1278207802F087F9304A304B127852
:104FD0000021207802F080F901222E4B1A702E4B0E
:104FE000DB78552B31D12D4B3B325A722C4B2D4A4D
:104FF000AB81EA812B826A822021307806F01CFC8A
:105000000120404205F0A0FD0120404205F03CFE99
:10501000FFF7C8F8FEF77CFE00F0B2FC012040422A
:10502000FEF752FF012006F0DFFCF02001F010FB3C
:105030000121307806F068FD307802F0E7FA1A486E
:1050400006F002FDFEF712FD70BD6422174B5B797E
:1050500053431A000A32CBE75862FF1F8D4D0011EF
:10506000914C00119843FF1FF461FF1F1462FF1F52
:105070002243FF1F6509FF1FADAC0000A464FF1FA2
:105080008264FF1F7842FF1F5942FF1F5664FF1FB3
:105090003764FF1F2864FF1F3862FF1F2C62FF1F49
:1050A000C4090000CE0900005A62FF1F3C62FF1FC6
:1050B000F8B50A0020230D001A40194263D05E4B58
:1050C0001B78002B5CD0FFF7D3FA5C4B5C4C5D4E39
:1050D00099686268737A8A1ADB039A4202D3616024
:1050E000FEF7C4FC327A217A531EDBB2994205D115
:1050F000FFF71AF9002000F0B3FD15E09142F9D353
:1051000000272772FFF74AF9A37ABB4202D0A772A1
:10511000FEF73AFD012000F0A3FD4B4F3800FEF7EB
:105120002FFE390006F0B8FD637A002B25D0013B35
:10513000DBB26372002B20D1444BDB78552B01D1BD
:1051400006F07AFCE37A002B12D00023A27AE372F5
:105150009A4202D0A372FEF717FD3D4A3A4F1388D8
:10516000380001331380FEF70BFE390006F094FD82
:10517000642370795843FFF78DFD237A013323723E
:1051800020206840F8BD0BB2002B0ADA314B1878AA
:1051900006F08AFC002801D006F01EFB80200002E9
:1051A000EFE70224214206D0254B01201A72FFF7B7
:1051B00085FE2000E5E70B071ED5FFF759FA1F4BC8
:1051C0001F49204C98684A68637A821ADB039A4226
:1051D00002D34860FEF74AFCFFF7E0F8FFF7A4F8B7
:1051E000012000F03DFD00F0E5FB2368DB0701D561
:1051F000FEF762FF0820C4E7CB0609D5FEF7C4FC22
:105200000D4B1B78002B01D1FEF796FD1020B8E75F
:105210000124214207D0104800F06CF806F0DCFCB5
:1052200000F004FDC5E70424080020402142A9D075
:10523000FEF766FEBDE7C0465A64FF1F4862FF1FC7
:105240002C62FF1F3C62FF1F5942FF1F3862FF1F85
:105250002062FF1F5862FF1F3C42FF1FF0B51B4B2F
:105260001B4F1B883A8804001A4E1B4D85B09A428A
:105270000DD832889A420AD3184B1A882B889A4242
:1052800005D1174A174B12881B889A421BD005205C
:1052900001F034FA3B8802AA1380338801905380CE
:1052A0002B88114D93800F4B02A91B88D3800F4B85
:1052B0002A78188802F050FF0D4B08212878019AAF
:1052C0001C7006F0C9FA05B0F0BDC0462664FF1F89
:1052D0004E42FF1F4C42FF1F4A42FF1F2464FF1F24
:1052E0002264FF1F4842FF1F8264FF1F5042FF1FBE
:1052F0002064FF1F13B50C4B1C78002C11D1002823
:1053000001D00A4B18600A4A0A4B11780A4A1078F1
:105310000A4A01920A4A0092002205F0C1FA2000CE
:1053200016BD1124FBE7C0468164FF1F1C64FF1FEC
:105330008064FF1F7064FF1F8264FF1F5C64FF1F97
:105340006064FF1F10B5064B12201B78052B06D199
:10535000044B13221988044B187801F0ABFB10BDE5
:105360008164FF1F5042FF1F8264FF1F10B500249D
:105370000122114B52421870104B1C70104B1A80B6
:1053800002F044F904220F4B21001A700E480C322F
:1053900006F0D2FB102221000C4806F0CDFB0722BC
:1053A0000B4B1C600B4B1C700B4B1C700B4B1A7087
:1053B0000B4B1C7010BDC0468264FF1F8164FF1F31
:1053C0005042FF1F8064FF1F7064FF1F6064FF1F57
:1053D0005C64FF1F3664FF1F3564FF1F5242FF1FCE
:1053E0003464FF1FF8B5174C0600257806A814246E
:1053F0000078052D23D1B41F134FA5B21824BD4248
:105400001DD88D1FADB2BD4219D8FA256D00AA4234
:1054100015D21D000D4F0A3DADB2BD420FD80C4C48
:1054200026800C4C21800C4900240A800B4A1380F2
:10543000FFF714FF0A4B0421187806F0F5FA200054
:10544000F8BDC0468164FF1F790C0000750C000098
:105450004E42FF1F4C42FF1F4A42FF1F4842FF1FA0
:105460008264FF1FF0B50BB20D0089B0002B00DB8A
:1054700070E1A44E307806F017FB041E50D003787C
:10548000A22B00D122E1D02B1AD0912B45D1437809
:105490000E2B42D19C4B82889A423ED19B4A836814
:1054A0001278052A39D1032018567F2835D0984B19
:1054B0001B68002B31D05B68002B2ED098472CE066
:1054C0008078072829D806F0CFFB0428183F3F74BE
:1054D000A8D86378002B0CD101218C4B19708D4B0F
:1054E0001A78002A5BD08C4B307801F0F5FE00284A
:1054F00055D00722854B1A7051E061780029F8D108
:10550000E378002B11D0854A854B1278307801F072
:10551000E3FE60706378002BEBD1200006F05CF9AD
:1055200080200002684009B0F0BD784B1B78022B48
:10553000F3D00121307806F02FFC0028EAD10121B8
:10554000307806F0E1FAE5E76378002BD1D16F4FB0
:10555000032807D13B78052B02D101333B701EE0B5
:105560000223FBE76F4B1A886F4B0293002A0BD084
:105570001B78002B03D00121307806F06DF93B78C1
:10558000062B04D1013BE9E7029B1A70F7E7042BD5
:1055900041D10121029B3078197006F0B5FA5C4BBD
:1055A0001B68002BB9D01B68002BB6D0574A107867
:1055B00084E76378554F002B27D10622211D5B48D5
:1055C00006F00AFC62895A4B5A491A80A2895A4B42
:1055D0001A80E3890B800521397058490A80584A9E
:1055E0001380228A574B1A80574B1B78012B09D105
:1055F0001F2001F083F8FA22920042430421307800
:1056000006F02AF90022484B75E7312B00D070E7ED
:105610000022454B1A700323A0E7062200214348CD
:1056200006F08AFA0023454A04211380444A307860
:105630001380444A138006F0F7F90821307806F009
:10564000F3F9A379083B5A425341304A03331370AC
:10565000304B1B78002B06D0334B30781A78002A59
:1056600006D001F077FE0122314B52421A8096E7B4
:105670000121197006F048FAF5E70821307806F0A4
:10568000D3F96378002B00D047E72C4B2D4F0293C2
:10569000E388029A04211380294B307803932389ED
:1056A000039A138063893B8006F076FB002800D0C4
:1056B00033E7264B1B68002B00D12EE70399029895
:1056C0003A88098800881B68984726E74379132B96
:1056D00000D022E70389012B0AD11D4B1B78022B36
:1056E00006D10821307806F09FF9FFF72BFE14E76A
:1056F000052001F003F808210200307806F0ACF82C
:105700000BE7C0468264FF1F051400008164FF1F81
:105710001C64FF1F7842FF1F5942FF1F5664FF1F82
:105720003764FF1F5864FF1F5A64FF1F2964FF1F5F
:105730005042FF1F3064FF1F3264FF1F2664FF1FAB
:105740002464FF1F2264FF1F2864FF1F1864FF1FCB
:105750002064FF1F8020C001014200D0E2E6CB0799
:1057600031D5324B1B78002B1DD0314E05AC337830
:10577000052B1AD1023B23702E4B21001B7823727C
:105780002D4B1B7863722D4B187801F049FD0028D2
:1057900009D007202A4B30701B68002B03D01B68F0
:1057A000002B00D098470120BCE60E20254B062296
:1057B0001B7825492370254B1B78637002ABC018FA
:1057C00006F00AFBD8E7022308001840194209D066
:1057D000174B1B78052B03D11D4B188806F04CF88E
:1057E00002209FE60424214203D0FFF737FD20006A
:1057F00098E6082308001840194200D193E6154B9B
:105800001C78012C03D0022C0DD008208AE6124B04
:10581000124A134913481B8812880988008800948B
:10582000FFF7E0FDF1E7FFF78DFDEEE75A64FF1F9C
:105830008164FF1F5242FF1F3464FF1F8264FF1FF9
:105840001C64FF1F3664FF1F5342FF1F3564FF1F98
:105850005042FF1F2064FF1F4842FF1F4A42FF1FA4
:105860004C42FF1F4E42FF1F10B502A804880B20B8
:10587000002C10D1496808784978090201430C4886
:10588000814209D1022119800A4B59881170DB78B5
:1058900000205BB2537010BD074C0A20A142FAD120
:1058A00002211980034B998811705B79F0E7C0469B
:1058B0006E2A00002062FF1F6F2A0000F7B5150056
:1058C00008AA16884A680F4F1478527812022243A9
:1058D0000A24BA4214D10122DBB2019200962A00B6
:1058E00005F0E4FE041E0BD1074B1B68002B07D00C
:1058F00068782A78000210434242504101309847AC
:105900002000FEBD022900009464FF1F30B5012570
:1059100003790400BFB02B4225D01449408805F01C
:1059200031FA28420CD0124B01A95B8D00220B806A
:1059300002234B800F4B5B888B80608802F002FB58
:105940000D49608805F01EFAC0070CD50B4B01A964
:105950001B8800220B8002234B80064B9B888B8088
:10596000608802F0EFFA3FB030BDC0468C64FF1F84
:105970007C42FF1F2062FF1F8464FF1FD642FF1F6F
:1059800010B5074C0749200005F0B2F92000064980
:1059900005F0AEF90721054A054805F06BF910BD81
:1059A000FFFF00008C64FF1F8464FF1F30BF0011E5
:1059B0007C42FF1F10B5024803F046F910BDC046F7
:1059C0000D59001170B540253F2608210B4BC20729
:1059D000D2172A40DD789C7835408C432A439C704E
:1059E000DA70820701D521439970400704D58022DF
:1059F000D97852420A43DA7070BDC046F442FF1FA4
:105A000013210A4BDA788A43123901400A43DA70CB
:105A10000222104202D0D9780A43DA70400703D537
:105A20001022D9780A43DA707047C046F442FF1F4B
:105A300010B5054B082419790A00A243002801D0AB
:105A400022000A431A7110BDF442FF1F10B5054B26
:105A50002024D9780A00A243002801D022000A435A
:105A6000DA7010BDF442FF1F0821F8B5324D334BF8
:105A7000AE7804000E40AE70984204DD67232B70B0
:105A8000273B6B70F8BD2E4B984203DAE0232B7056
:105A90001A3BF6E700232B706B7083B21A0029487B
:105AA0005F3292B2284F82422CD9002C03DA5B423B
:105AB0001CB204232B70053420B20A2105F0C4FE69
:105AC00004B2FA239B009C4232DB08232A7813435A
:105AD0002B706421200005F0B7FE0A2100B205F00A
:105AE000DBFF09B22A787B5C13432B700A2120006C
:105AF00005F0AAFE0A2100B205F0CEFF09B27B5CD8
:105B00006A780AE06970002CDBDA5B421CB204237D
:105B10002B70F5226B78092CE8DC13436B700A219B
:105B2000200005F0B9FF09B27B5C1E43AE70A9E707
:105B3000632CCEDCEDE7C046F442FF1F1B4E000095
:105B40001DFCFFFF2A0800005BBF00110823F7B50A
:105B5000194FCD003E7904001E403E71EDB263281E
:105B600006DD5F3333433B7140231D437D71F7BD39
:105B70000300093305DA20235B4233433B71C6231C
:105B8000F3E70E4B019300280BDA0423444224B2BE
:105B90003B710A21200005F07FFF019B09B25B5C8D
:105BA000E3E70928F5DD0A2105F04EFE019B00B26E
:105BB0001B5C1E433E71ECE7F442FF1F5BBF00110C
:105BC000F8B50A4F05003B780E00002B0CD0084CAE
:105BD0002000FEF727FC33002A0020003978FEF76A
:105BE00012FD2000FEF75CFCF8BDC0469864FF1F64
:105BF000FC42FF1F70B50A4E0A4D062231002800F4
:105C000005F0FAFD002809D0074C310006222800D3
:105C100006F0E2F807212000FFF7D2FF70BDC04672
:105C2000F442FF1FEE42FF1FED42FF1FE62220213C
:105C300010B50A4B1A70203A5A701C329A70DA78F2
:105C40000A40DA70082219791140353A0A431A716C
:105C5000F5225A71FFF7CEFF10BDC046F442FF1F78
:105C600010B5244B5B78002B3AD1002838D0224C59
:105C70000223E05E214B1B685B0632D509233221EB
:105C8000584305F0E1FD4130FF3000B2FFF7ECFE74
:105C90000520FFF797FE0422A35E194A6320934272
:105CA00005DC32331800642105F0CEFD00B201217D
:105CB000FFF74CFF237A0024132220009A42604110
:105CC000C0B2FFF7C3FE2000FFF79AFE0D4B187815
:105CD000053843425841C0B2FFF7AAFEFFF78AFFDA
:105CE00010BD0A21053005F0AFFD00B2FFF7BCFE84
:105CF0000320CEE73862FF1F2062FF1F3C62FF1FB8
:105D0000DD2600008164FF1F70B500250A4C2000CD
:105D1000A571FEF787FB11233E212000074AFEF7FD
:105D200072FCA84200D13E35054B20001D700123B6
:105D3000A371FEF7B5FB70BDFC42FF1F4ABF001107
:105D40009864FF1F0200F0B501270A480A4E511857
:105D50008B1A002B00DCF0BD08241578430868403E
:105D600038404000805B013C58406D08002CF5D164
:105D70000132EDE7FFFF00006CBF0011F0B5002518
:105D80000F269D4200DBF0BD4C5D070944403440C6
:105D9000A400A05801357840F3E70000F0B589B0C1
:105DA0006A460D000B000F27110010351C780133D7
:105DB000260024093E40167054700232AB42F5D1E1
:105DC0002023024AFFF7DAFF09B0F0BD70BF0011CF
:105DD000F0B54E780B7889B036020C0017000190B0
:105DE0001E43012A61D9954B9E4200D877E00133CA
:105DF0009E421CD1062A17D1CA788B7812021A4308
:105E00000B791B0413434A7912061A438C4B5A61CF
:105E100000221A705A808B4A5A608B4A9A608B4AC9
:105E2000DA60002009B0F0BD88225205EEE7884B09
:105E30009E423CD182498B78002B00D0F6E00C2AA0
:105E400031D10F22A3789343E278120213432279CF
:105E5000120413436279120613434B60E279A0796E
:105E600012020243207A00041043627A12060243AF
:105E7000CA60E27AA07A1202024376484A818342DB
:105E800008D804236E49142201980B7005F0A4FF72
:105E90001420C7E71201D21889235B059A42F0D873
:105EA00001238B70BDE7022AFAD00523EAE76A4A8C
:105EB00001239642E6D1FFF745FA052F0CD9E37886
:105EC000A2781B021343227912041A4363791B063A
:105ED0001343624A0393136005F0AEFDA1E7584DEA
:105EE0002B78002B9DD1AB78002B00D1A0E02B8923
:105EF00001339BB20093B34200D091E0132AD4D96E
:105F0000CF7C8B7C3F02122120001F43FFF71AFF3A
:105F1000874200D08EE0002E3DD1E378A2781B02AC
:105F200013432279E96812041A4363791B06134369
:105F300003930A228B4212D1FF23A370E3702371D3
:105F400063716B89002B09D1E37B227C1B02120455
:105F50001343A27B13431B0901336B8100226B891E
:105F6000002B8ED0002A67D1686837013818000BE3
:105F70006B6900030390984205D9686105F0C4FC81
:105F8000EB780133EB7068681022A11C381805F01B
:105F900043FD2E8145E76F89009A7B1E9BB2934299
:105FA0003AD1E278A37812021A43237905A81B0498
:105FB000134362796C6812061A43EB6800920392ED
:105FC000211D0C22049305F007FF0120260004A9DF
:105FD00040421036FFF7E2FE013F012F17D1009A31
:105FE0000B232861824200D04CE704221C49200088
:105FF00005F012FD042203A9686805F045FDE96873
:10600000039AFF23914200D13CE7F73B3AE7310086
:10601000FFF7C4FE1036DFE70923B742A4D831E703
:10602000009BB34200D9FCE607232BE7022329E7B4
:10603000032327E7062325E70A2323E7FFFE0000C3
:106040000443FF1F00000111FFFF000050485936B4
:1060500001FF0000FFFF001102FF000034F00040CC
:106060001043FF1F10B5034C0B000122210000F06C
:106070006BFA10BD256200110B8870B506000D008B
:106080000224162B11D92B000322094900F05CFAD7
:10609000041E0AD1074B2A881B88191C934200D979
:1060A000111C300089B200F0EFFA200070BDC0462C
:1060B00051620011AA64FF1F10B54A780400013A2A
:1060C0000B000220012A07D80A78002A04D00522F2
:1060D0002000024900F038FA10BDC0467F6200116E
:1060E0000A7810B50B0004000220002A04D0072211
:1060F0002000024900F028FA10BDC0462B630011B1
:106100000A7810B50B0004000220002A04D00922EE
:106110002000024900F018FA10BDC046916300113A
:1061200010B5034C0B000B22210000F00DFA10BD3E
:10613000C163001110B5034C0B000D22210000F0CB
:1061400003FA10BD3364001110B5034C0B000F228D
:10615000210000F0F9F910BD8D6400110A7810B526
:106160000B0004000220002A04D011222000024962
:1061700000F0EAF910BDC0469D640011002310B57F
:106180001322190000F0E0F910BD000010B5034C17
:106190000B001722210000F0D7F910BDEF640011A9
:1061A000002310B51922190000F0CEF910BD00002F
:1061B00010B5034C0B001B22210000F0C5F910BDE7
:1061C00029650011F7B584890D0006000121002C16
:1061D00022D000238268D3561778002B1EDA0C2CAD
:1061E0001AD90C3CA4B2131940880093230002F082
:1061F00086FE431E984101307B06DB0F6B703F2308
:10620000013C1F40A4B22870AF70AC80002C07D0B6
:10621000B3680133AB6000210800FEBD0020EBE74E
:10622000AC60F8E70B7803704B8843704B881B0A0F
:1062300083700B79C370042070470420022B06D1B1
:106240000020537811781B02009A0B43138070478B
:106250000B8803700B881B0A4370022070470420D0
:10626000009983420AD1537810781B0203430B80B4
:10627000D37890781B02034300204B807047F8B519
:106280000D004B7801240021461C03702B788B42B3
:1062900001D82000F8BD6B78B01C4F1C012B10D129
:1062A000890069184B88022233704B88B9001B0A99
:1062B0007370691805F0F8FC04360434A4B2F9B21E
:1062C000E4E7122359436B185A88043132705B8813
:1062D00010221B0A7370691805F0E6FC123612349E
:1062E000ECE770B5049D14001E00052B01D80420B6
:1062F00070BD637812781B0213432B80E378A27879
:106300001B02134302226B802A71211D681D063E69
:1063100005F0CAFCB2B22A81E92AE8D82800A11DFA
:106320000A3005F0C1FC0020E2E7002310B50A782E
:106330009A4201D8900010BD9A008A1854880133FF
:1063400004705488DBB2240A447094888470928864
:10635000120AC2700430EAE710B51100029C062B45
:1063600004D004201022142B01D010BD022222716F
:106370004B7808781B0203432380CB7888781B0274
:10638000034363800431601D05F08EFC0020ECE7C0
:1063900010B50C788B7804315C43E4B203702200B2
:1063A000013005F081FC601C10BD0420022B06D1D9
:1063B0000020537811781B02009A0B43138070471A
:1063C00010B50C000A88023105F06EFC208810BD63
:1063D00070B504000D0004981100012B01D80420B1
:1063E00070BD167852781202324302800200F132F8
:1063F00055701470E125002C00D10C35023B9AB287
:106400004280AA42EBD80231043005F04DFC002056
:10641000E6E70420009983420AD1537810781B02E2
:1064200003430B80D37890781B02034300204B80FA
:10643000704710B50C000A88023105F035FC208841
:1064400010BD000070B501211E000420049C0E4008
:106450000B4218D1CB40DDB28D4214D90A49DBB2D0
:10646000098899420FD32300EE331D703300580082
:1064700011184978165C0902314301332152D9B20F
:106480008D42F4D8002070BD1C43FF1F10B50C00D6
:106490000A88023105F008FC208810BD10B50C7880
:1064A0008B7804315C43E4B203702200013005F0C4
:1064B000FBFB601C10BD10B511000298032B01D826
:1064C000042010BD14785278043B1202224302804B
:1064D000CA788C781202224342809AB28280EB2AD8
:1064E000EED80431063005F0DFFB0020E9E710B5F7
:1064F0000C000B8803700B881B0A43704B88837059
:106500004B881B0AC3708A880430063105F0CCFB27
:10651000A088043080B210BD0420012B03D10020DC
:106520001378009A1370704710B50C000B88037035
:106530000B881B0A43704A880230043105F0B4FB13
:106540006088023080B210BDF0B589B003931E4B55
:10655000029242000700D05A019102F020F8132560
:10656000061E2DD0029B01240370019B002B04D03A
:10657000001903999847001984B26B461B7A5BB2E5
:10658000002B0FDA1021380002F01CFB192500281F
:1065900013D130003219E1B202F066FC051E0CD1B5
:1065A0000C34A4B2042304AA380005A993800696EB
:1065B000948101F0AFFD051E02D0300005F08CFA89
:1065C000280009B0F0BDC046A864FF1F70B50500E3
:1065D0000C0000280CD00020814209D0102220009D
:1065E000044905F061FB01202B7823736B786373FA
:1065F00070BDC046B0BF0011F0B506000D00170019
:106600001C0085B002291BD00020102907D1022BC5
:1066100007D0102B03D115E00020102C08D005B0B6
:10662000F0BD69463800FFF7D1FF2A0069460BE04C
:1066300069463000FFF7CAFF22006946380004E0CF
:10664000022BE9D12A003900300005F09DFAE6E777
:10665000031CF02800D9F023032008499AB2013A1C
:106660000B80D317034006499B189B100B80D30F58
:1066700004499B185B100B807047C0462043FF1FE6
:106680001E43FF1F1C43FF1F034B1B888B4202D37B
:10669000024B4000C15270472043FF1FA864FF1FF8
:1066A000014B4000185A7047A864FF1F1722014B86
:1066B0001A807047A864FF1F70B505000E2005F012
:1066C0007BFB041E13D0D0230370002306228370AB
:1066D00007494570033005F0E7FA064B2100DA8AD6
:1066E00062811B7E2373044B187805F06DF870BD32
:1066F000C464FF1FB464FF1F7043FF1F262803D824
:10670000024B4000C05A70470148FCE72243FF1F7C
:10671000FFFF000070B506000C00094D1C2200218F
:10672000280005F009FA074B1E70074B1C7005F096
:1067300063FA0123002801D0002312202B7070BDC2
:10674000B464FF1F7043FF1FD564FF1F70B50500C1
:106750000D4C0800E260A16010220021656005F088
:10676000DBF9012803D11021A06802F058FD1022A6
:106770000021280005F0D0F9012803D1102160681C
:1067800002F04DFD70BDC046B464FF1F70B5041E1D
:1067900005D1002903D006220D4805F085FA0D4BDE
:1067A0001D78012D11D1002C05D102221A7005F09F
:1067B000CBF9280070BD00221A70074B1B78FF2B05
:1067C000F7D02000FFF778FFF3E70025F1E7C04698
:1067D000C464FF1FB464FF1F7043FF1F030010B5A4
:1067E000002801D1002010BD00780B4A002803D1F9
:1067F0005988D1821B7913761378022BF2D10023AA
:10680000984200D103331370044B1B78FF2B01D047
:10681000FFF752FF0120E6E7B464FF1F7043FF1F3C
:10682000002911D000280CD04B79012803D1402237
:106830005242134303E03F221340032802D00120B9
:106840004B7170474022F4E70800FAE770B5094D34
:106850000100287800280BD0074C0622200005F004
:1068600023FA21002878FFF7DBFF200005F09CFACF
:1068700070BDC046D464FF1FAE64FF1F00290AD05C
:10688000012808D13F224B799343C02B03D0403BD2
:106890005A425341981C704770B5174D06002B782B
:1068A000FF2B15D00A2005F087FA041E10D0D02344
:1068B0000370C83B8370114B11491B784670C3703D
:1068C0000622043005F0F0F92100287804F07CFF5E
:1068D0000C4B1B78012B0DD10B4B1B68002B03D0ED
:1068E0009B68002B00D09847084B04211878084A71
:1068F00005F04AF870BDC0467043FF1FD464FF1F07
:10690000AE64FF1FD064FF1FFC64FF1F0065FF1F04
:1069100060EA0000014B98687047C046B464FF1FEE
:10692000014BDB6818687047B464FF1F074B10B554
:10693000DA68136801331360054B1878FF2803D019
:106940008021C90105F0E0F810BDC046B464FF1F06
:106950007043FF1FF7B50E0002F0C8F8051E1CD0EB
:106960000E4B06621F78002F00D10778AB791020FC
:10697000019305F021FA041E0FD0D0230380C73BFA
:106980008370019BE91DC3700622043005F08CF969
:1069900021003800E66004F017FFF7BD6E43FF1FCB
:1069A000014B18787047C046D464FF1F054B002880
:1069B00005D1054B1A78054B002A00D1014B180070
:1069C0007047C046C464FF1FD464FF1FAE64FF1F3E
:1069D000014B58687047C046B464FF1F024B1868EB
:1069E000431E9841C0B27047D864FF1F421E030087
:1069F0000120152A03D9FF3B5A425341D8B27047B0
:106A0000F0B51C0000230E0085B0039002920B70BD
:106A1000029A934201D3002019E0E55C5A1CD2B2DD
:106A2000002DF8D0029851198142F4DC0233DFB214
:106A3000A35C18000193FFF7D9FF002807D0013DA0
:106A4000019A0399EBB233708A4202D1E01905B082
:106A5000F0BDDB19DBB2DBE710B50C0002F09EF8ED
:106A600003001220002B03D02100588805F03CF9C8
:106A700010BD000070B50E4D84006359002B15D079
:106A8000186A002801D005F017F92B59586A002818
:106A900001D005F011F92B59986A002801D005F0B2
:106AA0000BF9285905F008F900232B5170BDC04699
:106AB000E464FF1F1C4B70B504000E0015009942E2
:106AC0000AD11A4B1B68002B01D1122070BD1B6824
:106AD000002BFAD09847F9E7154B994215D1134B83
:106AE0001B68002B0AD01B68002B07D09847002892
:106AF00004D1104B1C70104B1D70E7E729002000DB
:106B0000FFF7AAFF0028E1D1F3E7080001F0EEFF4C
:106B10000028DAD003780320A342D7D1290030001F
:106B200005F0E2F8D2E7C046FEFF0000E064FF1F78
:106B3000FFFF0000DD64FF1FDC64FF1FF7B50400EA
:106B4000808801F0D3FF0025A84203D00578A088F3
:106B500002F008F81C4E3378002B1FD0AB421DD139
:106B60001A4B28001978FFF777FF002818D0002368
:106B70003370A3790820A778A688019305F01CF943
:106B8000011E0DD0D0230370CA3B8370019B477058
:106B900086808371280004F017FE01E0002DE8D103
:106BA000A0880B4B8200D358002B01D0FFF762FF67
:106BB0001721A088FFF768FDA08801F027FDA088B5
:106BC00001F0FEFDF7BDC046DD64FF1FDC64FF1F62
:106BD000E464FF1FF0B587B01D000CAB1B880700F5
:106BE00001930DAB1B88142002930EAB1B8816007B
:106BF00003930FAB1B880091049310AB1B88059384
:106C000005F0DAF8041E1AD0D0230370CB3B47708E
:106C10008370C670062229000430002D11D005F0C3
:106C200043F8019B21006381029B0098A381039B91
:106C3000E381049B2382059BA37404F0C5FD07B088
:106C4000F0BD04F079FFECE7F7B5009308AB1B88C3
:106C500007000C200D001600019305F0ADF8041E8E
:106C600013D0280001F042FF00280FD00078D02375
:106C70002370C93BA370009B21002381019B677097
:106C8000A580E680638104F09FFDF7BD014B187875
:106C9000EDE7C0467043FF1F13B504006489038904
:106CA000C2888188C0780094FFF7CEFF13BD000032
:106CB00010B5044C2068002803D004F0FDFF002329
:106CC000236010BDE864FF1FA122F0B58188920007
:106CD0004A43384B384F1B6804009B189D22920092
:106CE0009B18827989B01A603B68002B5FD01D78B1
:106CF000324B1B68002B04D05B68002B01D00020B6
:106D00009847260008363100E079FFF7B7FD237D6C
:106D1000E0710200E0780493638A29000393238AD8
:106D20000293E3890193A38800933300FFF752FF96
:106D3000E378002B0BD1E289A379A1880292019616
:106D4000E27928000092012201F0DAFEE0703B684F
:106D5000002B20D0FFF7ACFF194D287800281AD05F
:106D6000184B1978FFF778FE002814D02B78E678B6
:106D700008200793A78805F01FF8011E09D0D0232B
:106D80000370CA3B4670837087808671079804F051
:106D90001BFD00232B701721A088FFF775FCA0882E
:106DA00001F034FCA08801F00BFD09B0F0BD064BEA
:106DB0009DE7C0463409FF1FE864FF1FFC64FF1F06
:106DC000DD64FF1FDC64FF1F7043FF1FF8B5070081
:106DD00008000E0001F08AFE041E18D02620FFF7DE
:106DE0008DFC051E00D12578062004F0E5FF041E69
:106DF0000DD00021062204F09FFED0232370C23B59
:106E000021006770A370A680E8B204F0DDFCF8BD35
:106E1000F0B585B001930AAB1B78070002930BAB6A
:106E20001B7808000D000092039301F05FFE061E20
:106E300022D0102004F0C0FF041E1DD0102200211B
:106E400004F07AFE2620FFF759FC002800D13078A4
:106E5000D0232370C13BA370009B21002372019BB0
:106E600067706372029BA580A372039BC0B2E3723A
:106E70000C9BE36004F0A8FC05B0F0BDF7B50D0075
:106E8000019001F033FE071E20D00E2004F094FF85
:106E9000041E1BD02620FFF731FC061E00D13E78D1
:106EA000D0232380C53B0622A370F91DE01C04F00B
:106EB000FBFE019B2A0063810123DD401A401D4037
:106EC000210022736573F0B204F07EFCF7BD000070
:106ED000F0B585B0029010000D0017000A9E0393D4
:106EE00001F004FE041E31D0029B002B2ED1039B27
:106EF00002795B0724D5122313430422002E08D104
:106F00000B99002905D10C99002902D10D9900296E
:106F10001AD01A430D9B2271002B00D0C9E0002E1D
:106F200000D1CFE0002D00D0CCE0606A002801D075
:106F300004F0C2FE1C21300004F0C6FC606205E0D3
:106F400002239A430E33D7E793432371654BBA006C
:106F5000D458002C00D1AAE0002E10D0236A002BB8
:106F600003D11C2004F028FE20625E4BBA00D358E7
:106F7000186A002803D01C22310004F095FE0C9BF7
:106F8000002B12D0574CBB001D596B6A002B03D14C
:106F9000162004F011FE6862BB00E358586A00280E
:106FA00003D016220C9904F07FFE0D9B002B11D00C
:106FB0004C4DBC006659B36A002B03D1142004F079
:106FC000FBFDB0622B59986A002803D014220D995A
:106FD00004F06AFE380001F089FD051E67D0414BC0
:106FE000BA00D358002B62D01A6A3420002A00D18C
:106FF0001C389A6A002A01D0143080B20B9A002AF9
:1070000001D01C3080B25B6A002B01D0163080B2F8
:1070100004F0D2FE041E4AD01822002104F08CFD98
:107020002620FFF76BFB0190002801D12B780193FC
:10703000D0232370029B200063700A23294EA37083
:10704000039BBD00A371AB59A780196A18300029B2
:1070500005D01C22A06004F027FE200034307359B4
:10706000996A002907D0030014221433E0600293C8
:1070700004F01AFE02980B9B002B08D003001C2280
:107080001C330B992061029304F00EFE0298735991
:10709000596A002903D01622606104F005FE6B4690
:1070A0002100187904F090FB3800FFF7E3FC05B0ED
:1070B000F0BD10220D9B0D991B69A018236204F0EE
:1070C000F3FD2CE70B9B002B00D13FE7012D00D0F7
:1070D0003CE7606A002801D004F0EEFD1C210B980B
:1070E0002AE7C046E464FF1F10B5044C206800285E
:1070F00003D004F0E1FD0023236010BDD864FF1F1E
:107100000B4B07B51A68002A01D100200EBD694655
:10711000531C012012780731FFF772FC0028F4D0CD
:1071200002780123100018401A42EED0EEE7C04664
:10713000F464FF1FF0B51F4F01203B6887B0002BA0
:1071400025D09B78059300F0B3FB002821D00A20BE
:10715000FFF7D4FA04000B20FFF7D0FA164B050016
:107160001E78731E9E413B68F6B2191DD878FFF752
:1071700057FB3B682900DA7A043303929A7901932A
:107180000292009033002000059A04F03DFC07B005
:10719000F0BDFFF7B5FF002805D00620FFF7AEFAD7
:1071A00004000720D8E70820FFF7A8FA0400092008
:1071B000D2E7C046D864FF1FD464FF1F70B50A4EE3
:1071C000040033780D00FF2B0DD0042004F0F4FDF3
:1071D000011E08D0D0230370CE3B45708370C4706D
:1071E000307804F0F1FA70BD8043FF1F70B50400E1
:1071F00006200D0004F0E0FD011E0AD0D02303702C
:10720000CD3B8370054B44701B688580187804F073
:10721000DBFA002C01D0FFF767FF70BDD864FF1FB9
:10722000F8B5264F06003B680D001124002B05D150
:107230000522234B1B78134202D112242000F8BDF3
:10724000204A10241268002AF8D01278002AF5D0BB
:10725000DB0719D52B789A1E012A1AD80C2004F0C6
:10726000ABFC132438600028E8D000230A224370C6
:1072700029000670023004F017FDFFF75BFF041EC3
:107280000AD0FFF731FFD9E700F012FB0028E1D167
:10729000E4E7002BE2D0D0E70B4B1B78032BCDD1DA
:1072A0001D20FFF72BFA094B18800028C6D0084B89
:1072B00004211878074A04F067FBBFE7D864FF1F72
:1072C000D564FF1FF464FF1FD464FF1FD264FF1F47
:1072D0000065FF1F60EA0000F7B50193194B140029
:1072E0001A78052306000F0012201A4221D0012926
:1072F00020D1154B1D68002D1BD002201F2C18D843
:10730000002C02D0019B002B13D0104B1F221E70AB
:107310006E1C0021300004F00FFC019922003000A7
:1073200004F0C2FC310020002C70002F06D004F0C5
:10733000CBFCFEBD064B12201D68DCE704F0A4FA6E
:10734000F7E7C046D564FF1FF464FF1F8043FF1FAB
:10735000F064FF1FF8B50F4E12243368002B17D0CE
:107360001B780F3C834213D100250B4F0221387844
:1073700004F05AFB094B042138781D8004F054FBBB
:10738000074B28001D8033685C7004F01DFB04006F
:107390002000F8BDD864FF1F0065FF1FEC64FF1FCD
:1073A000D264FF1F70B5012823D11B4C2388002B0A
:1073B00003D01A4A1578002D07D0194B1B68002BF3
:1073C00002D01878FFF7C6FF70BD3B2B02D93C3BBB
:1073D0002380F9E7134E0221307804F025FBFA22CE
:1073E0002388920002215A43307804F035FA258030
:1073F000EAE70B4B1B68002BE6D00B4B1B785B07B7
:10740000E2D5084B0221187804F00EFB0022024B53
:107410001A80FFF769FED7E7EC64FF1FD064FF1FF7
:10742000D864FF1F0065FF1FD564FF1FF8B51E4D10
:107430002868002803D004F03FFC00232B601B4E7B
:107440003068002803D004F037FC00233360184F65
:1074500005243B7818002040234221D0154800F035
:107460002BFA3B78234213D0202004F0A5FB2860A0
:10747000002813D02022002104F05EFB202004F01D
:107480009BFB041E306005D02022002104F054FB39
:10749000002004E0286804F00FFC2C601320F8BDE5
:1074A00000F00AFAF4E7C046F464FF1FF064FF1F1F
:1074B000D564FF1F7443FF1F10B50A4C23681A1EC2
:1074C0000ED0002808D10130587004F07DFA002851
:1074D00005D02368002B02D00021FFF787FE012290
:1074E000100010BDD864FF1FF7B5274E05003368A4
:1074F0000191181E21D05C78244F012C30D1FFF768
:10750000FFFD002825D02000FFF7F8F804004128EF
:1075100014D91F4B022118781E4A04F035FA1E4B6D
:107520003C3C1C80022233685A703B78002B14D1FB
:1075300028000199FFF75AFE0120FEBDFA229200B1
:107540004243002AEED0124B0221187804F084F94D
:10755000E8E7FFF7D3F80200F3E700233B70EBE71F
:107560003B78002BE8D1032004F026FC011E08D054
:10757000D0230370CC3B457083703368187804F0D7
:1075800023F9FFF7B1FDD7E7D864FF1FD064FF1FD1
:107590000065FF1F60EA0000EC64FF1F10B517498B
:1075A000838802008B4220D011D815498B4217D016
:1075B000144900205B1899B2012907D89268117804
:1075C0005A425341D8B2FFF7F9FD012010BD0E4ACF
:1075D00000209B1807229BB29A424041C0B2F5E7B7
:1075E00083681878FFF768FFF0E7836899785A781E
:1075F000090218781143FFF777FFE7E70A20000038
:1076000006200000F8DFFFFFAFDFFFFF014B18701F
:107610007047C0468143FF1F10B5064C207001F033
:1076200041FA207804F098F90521207800F062FDF5
:1076300010BDC0460065FF1F0BB273B50D00002BD7
:1076400000DBC4E0884B187804F02EFA041E0ED03C
:107650000378912B0FD0A22B00D1A1E0834B187897
:10766000FF2852D0210004F0AFF800284DD180202F
:107670000002684076BD43780F2B76D013D8052BD7
:1076800070D00E2BEAD18088794B98422BD8794B59
:1076900098421BD8784B9842E0D1A3681878591CBF
:1076A000FFF774F838E03E2BD8D18378032B74D0E1
:1076B0006CD8012B6ED0022BD0D1704B1B68002BE5
:1076C00023D05B68002B20D098471EE06C4BC0187D
:1076D0000C28C3D804F0B0FA1DC2C2150BC20B0BA4
:1076E0000B3223C23C00674BC0180728B6D8664B44
:1076F0001B68002B09D01B68002B06D02000984780
:107700000AE0A3681878FFF7C7F8200004F064F8CF
:10771000ADE7A068FFF762F800289FD0F5E7A368FF
:107720001B78002BF1D0554B1B68002BEDD01B684C
:10773000002BEAD0210055489847EDE74F4B1B68D6
:10774000002BE2D01B68002BDFD021005048F3E76C
:10775000504B1B68002BD8D05B68002BD5D0210084
:107760004348E9E7FFF7EAF9CFE780884A4B9842B8
:1077700003D04A4B984200D070E7464B1B68002B61
:10778000C3D05B68002BC0D02100D5E7153B012B8F
:10779000BBD963E7FFF798FAB7E7FFF77DFAB4E7DD
:1077A0003F4B1B78042B07D100236A4613800179D5
:1077B000408800F0C5FCA8E7364B1B68002BA4D01E
:1077C0005B68002BA1D00100364898479DE7012453
:1077D00021420AD0294B1B68002B04D05B68002B88
:1077E00001D000209847012043E78B070AD5264B9C
:1077F0001B68002B04D05B68002B01D02000984749
:10780000022036E70421280008400D4200D131E76C
:10781000254E3388002B21D0013B9BB23380002BB7
:107820001AD1FFF7DBF800280AD0204B1C70164B4A
:107830001B68002B04D05B68002B01D02000984708
:10784000FFF7C6F8694601F001FD6846FEF7FEFF46
:107850001D20FEF753FF308004200AE7024B187802
:1078600004F0E2F8F8E7C0460065FF1F8143FF1F00
:107870000E2000000120000009100000F864FF1F26
:10788000FEDFFFFFAFDFFFFFFC64FF1F0C200000E7
:107890000B200000E064FF1F0D20000013200000FB
:1078A000D564FF1FFFFF0000D264FF1FD064FF1FDD
:1078B00010B501F09BF910BD014B18607047C04630
:1078C000FC64FF1F0B880020162B01D8172304200F
:1078D000014A13807047C046AA64FF1F002070470A
:1078E000074A03001188814207D0918800209942FD
:1078F00002D101308000101870470020FAE7C0461E
:107900000865FF1FF0B58F7806000D00C5B01E2F6B
:1079100015D1FFF7E5FF051E03D10024200045B077
:10792000F0BD00223B003100C078009200F0B2FBB5
:107930000400A81C00F0D2FBFF23EB70EEE7264BFF
:10794000062403931B78FF2BE8D0182FE6D87B087A
:10795000224A013BDB0002929A589446002ADDD06D
:10796000029AD3185B68002BD8D00878002802D17F
:107970004B78012B02D10624122FCFD107AFAB8851
:10798000697800976446AA68A047041EC6D1AB7800
:10799000029A5B08013BDB00D318390030005B68BA
:1079A0009847041E0BD1AB78042BB6D0039A310054
:1079B00010782200009700F06DFB0400AEE76A78B3
:1079C000002AABD1AA7805A93B88087130000A705B
:1079D0004B80FEF747FBA0E78443FF1FC0BF0011A9
:1079E0001D4B37B5050098420BD000290AD1FFF78F
:1079F00077FF002805D11948FFF772FF002800D053
:107A0000058037BD01291AD1FFF76AFF041EF8D09F
:107A100001235B420380A378FF2BF2D0FE2B07D01B
:107A20000023E0781422009329001E3300F032FB7B
:107A3000A01C00F053FB01235B426380E1E70229B5
:107A4000DFD1013901F0BEF80028DAD12800FFF7B4
:107A500047FF041EDFD1D4E7FEFF0000FFFF000058
:107A6000022210B5074B52421A80074801325A8051
:107A70009A80DA8000F07EFA044801F025F80020B0
:107A800010BDC0460865FF1F05790011E17900119E
:107A90000388F7B50400002B02D102252800FEBDA3
:107AA00042680221137825485268FEF7A5FD002898
:107AB0002ED0234F01253A88002AEFD08023218839
:107AC0005B0201259B1A9942E8DC0C2004F074F853
:107AD000061E31D03B8822889C4600231800019561
:107AE00061469DB2491989B2AA421BD8002801D02B
:107AF00062443A8000233000082208C0210004F0CC
:107B0000D3F8104A1368002B13D100251660C5E77F
:107B10006268022113780C485268FEF76DFD002858
:107B2000C7D1BAE760681D0140194181013301984E
:107B3000D6E71A001B68E6E71325AFE72EC0001151
:107B40008243FF1F0465FF1F2CC00011014B1870FA
:107B50007047C0468443FF1F14230A0010B51A4023
:107B6000194204D00122102101F048F810BD4B0643
:107B7000F9D4012088434000F8E710B514008B06C3
:107B800004D50122102101F039F810BD08230A00A4
:107B90001A40194202D14BB2002B0FDA102101F02A
:107BA0002DF8002808D02300F2331B78002BECD0EE
:107BB000F1342378012BE8D10020E6E70320890780
:107BC000FAD4E2E7F0B51F00184B85B01C680190AD
:107BD00002910392002C27D1200005B0F0BDA568CA
:107BE0003301ED186B89019A934211D3029A9342A3
:107BF0000ED8002F04D10A9B002B10D12C00EBE7EC
:107C00003B002978039A6868FEF7F6FC0028F2D159
:107C10000136B6B2A388B342E1D82468DAE7A36894
:107C20000A9A5B891380E9E70026F3E70465FF1FE2
:107C300037B50C000A8849880123914217D3002ADE
:107C400015D0651D23792A0002210A48FEF7D4FCCD
:107C5000102300280BD023796188208800242A0073
:107C60000094FFF7AFFF0A23A04200D023001800C2
:107C70003EBDC0462EC0001113B50A0008884988D1
:107C8000012388420BD8002809D00024137905323B
:107C90000094FFF797FF0A23A04200D023001800AA
:107CA00016BD13B50A0008884988012388420BD8FD
:107CB000002809D00024137905320094FFF782FFD1
:107CC0000A23A04200D02300180016BDF0B58BB0E7
:107CD00003904A8808880E000123824255D3002869
:107CE00053D00023012704AC2370002271881300B5
:107CF0000092FFF767FF051E3ED02078002835D19F
:107D00002B78022B18D167706A8983000130E31841
:107D100080005A8069680222201803F0C5FF23788A
:107D20000133DBB22370042B19D93B006889013081
:107D300080B2002BD9D01FE0022363701223584376
:107D40006A89231804305A8069681022201803F0C9
:107D5000ABFF23780133DBB22370002BE5D10C4A53
:107D60006B899B185A425341DBB2DFE76378012BE2
:107D7000E4D12B78022BC7D022780A23002A04D022
:107D800021000398FEF798F9002318000BB0F0BD0E
:107D90000100FFFF0F4BF0B504001868002816D053
:107DA00083685D89A54207D88288AE18B44203DA99
:107DB00012019A18934201D10068EFE71E005F8913
:107DC0001036A74204D1002900D00D801800F0BD64
:107DD0003300EFE70465FF1F70B505000C0008884D
:107DE0000021FFF7D7FF03000120002B04D0220061
:107DF0002800197AFFF7C1FE70BDF7B50C00002509
:107E000001902300EE331B78AB4201D800200AE03A
:107E10006B00E65A00213000E718FFF7BBFF00288F
:107E200002D126800130FEBD017A0198FFF794FE51
:107E3000002802D03B882380F5E70135EDB2E0E76A
:107E400010B5040008880021FFF7A4FF03000120FB
:107E5000002B03D02000197AFFF77EFE10BD000032
:107E6000054B1B68002B01D1180004E09A68528969
:107E70008242F6D1988870470465FF1FF0B50E273F
:107E8000002687B0039302ABFF183E8005001F4B0E
:107E900040891400984207D02B78013000976A6817
:107EA00080B2FFF78FFE060002212B7818486A681F
:107EB000FEF7A2FB00280FD06C892000FFF7D0FF4F
:107EC000002802D0013C0419A4B2039B002B00D06F
:107ED0001C80300007B0F0BD02212B780D486A6885
:107EE000FEF78AFB0028E7D102212B780A486A684E
:107EF000FEF782FB002807D0002EDED03B88A3428D
:107F0000DBD17489013CDFE76C89DEE7FFFF00000D
:107F10002EC000112CC000112AC0001110B50C0099
:107F2000FFF7DEFC03000220002B0AD0002C00D05B
:107F300023609B781720FE2B03D00138FF2B00D144
:107F4000002010BD73B50D0001A904001600FFF755
:107F5000E5FF172805D0002E04D129002000FEF7E8
:107F600027F976BD01221021200000F047FE0028ED
:107F7000F3D0F6E7014B18607047C0461465FF1F49
:107F800037B56B469D1D010004000222280003F056
:107F900023FF2B88B02B0ED12379122B09D123007C
:107FA000FA331B78012B06D10121608800F0E0F83C
:107FB00001E01B2BF8D037BD10B5054B042118701C
:107FC00000F098F8FFF74CFDFEF770FB10BDC046BF
:107FD0001865FF1F0020F0B50BB20F0087B0834279
:107FE00034DA274B187803F05FFD051E2BD0037899
:107FF000A02B25D103AE3100FEF7E4F8041E0BD10F
:10800000B378DB0724D51F4B06341B68002B03D045
:108010003100688898470400A868002801D003F060
:108020005BFD002C08D1184A039B1340174A93426A
:1080300006D0B3781B2B03D00121688800F098F894
:10804000280003F0C9FB80200002784007B0F0BD93
:108050000F4B1B68002B10D0310068889847041E16
:10806000DAD07378002BD7D1B27801A90A704B808F
:108070000C716888FDF7F6FFCEE70624F1E7C046ED
:108080001865FF1F1065FF1F00FFFF0000011200B1
:108090001465FF1FF7B50190FC200D0017001E00AE
:1080A00003F08AFE04001320002C12D0B02320001D
:1080B0002370089BF4226770658026710830002BBE
:1080C00008D0190003F0F0FD2100019803F07CFBBB
:1080D0000020FEBD089903F02FFDF5E710B5041E42
:1080E00006D00078FD2803D803F09EFBFF23237001
:1080F00010BD00000A1F93B210B504000220032B2C
:1081000005D882400020024BD1529B189C7010BDB4
:108110003865FF1F0B8870B5043B04000D0002207A
:10812000032B0BD80121200000F04CFD030014208C
:10813000002B03D02900200000F0DEFB70BD000002
:1081400007B51300034A00920A00012100F02CFC3D
:108150000EBDC0467D83001107B501920322009237
:10816000024B0A00122100F049FC0EBDFB830011F6
:1081700007B56B4601AA11800449D88008780633F8
:10818000012802D1190003F0DFFB07BD1965FF1FAD
:108190000C4B10B518700023FF210B4A138013817C
:1081A00093819380094A5380137051729381937223
:1081B000D174D3821375517703F0AEFD00F0FCF952
:1081C00010BDC0464865FF1F3865FF1F1A65FF1FB9
:1081D000F0B58DB06B46002003910C229B5E83426C
:1081E00000DBB0E05D4B187803F05EFC051E00D1AB
:1081F000A4E00378902B00D09DE006AF01004688F4
:10820000380000F013FA79680400002900D19CE0DE
:108210003B88052B6ED13B89032B1CD905AC200074
:1082200000F0A2F86288172A61D83989131D994293
:1082300031D17968237804310291D90738D5607833
:1082400000F08EF9071E06D0002303712378012B5E
:1082500008D0132B23D0A868002800D178E003F0C1
:108260003BFC75E06288029909A800F0A6F802902C
:10827000380000F08BF909AA2378387A019200229D
:1082800031000092029A00F012F9380000F064F90F
:10829000029B002BDFD0300000F080F9DBE7037891
:1082A000032BD8D16288029909A800F0D6F8DEE73E
:1082B000122B13D1029909A800F0B5F8021EEAD1D9
:1082C00027498B88002BC6D0887909A9237801918A
:1082D00061780091310000F0EAF8BCE7002302AABF
:1082E00093833000617809AAFFF72AFFB3E71D4B9B
:1082F0000993F6E7042B02D09A1F012AABD8184A3B
:10830000043B9B00995A0029A5D0D21890783100DF
:108310003A0000F0AEF800289DD13B88042B03D032
:1083200001213000FFF724FF012C04D1A8680028A8
:1083300001D003F0D1FB280003F04EFA8020039B0C
:108340000002434018000DB0F0BD012800D182E7C3
:1083500001213000FFF70CFFEDE7C0464865FF1F25
:108360003865FF1F010017000B7803704B784370CE
:10837000CB788A781B021343438070470A88030036
:1083800002700A88120A42700A88012A06D14A88B5
:1083900082704A88120AC27004207047022082420A
:1083A000FBD14A8804309A704A88120ADA708A88A7
:1083B0001A718A88120A5A71EFE710B50400012079
:1083C00082420CD94B780A781B02134323808342E4
:1083D00006D1CB788A781B0213436380002010BD3E
:1083E000022BFBD1CB788A781B02134363804B7935
:1083F0000A791B021343A380F0E70B8803700B88F4
:108400001B0A43704B8883704B881B0AC3708B8890
:1084100003718B881B0A4371CB888371CB881B0A3D
:10842000C3710820704703000120082A14D14A783C
:108430000878120202431A80CA788878120202432E
:108440005A804A790879120202439A80CA79887957
:10845000120202430020DA80704710B504000120A8
:10846000022A05D100204B780A781B02134323808F
:1084700010BDF8B5060010200F00150003F09CFC9D
:1084800004000120002C0ED0A0230C222900238000
:108490006780201D002D07D003F006FC210030006E
:1084A00003F092F90020F8BD03F046FBF6E7F7B5BC
:1084B0001E00009008AB142017001D78019103F0F6
:1084C0007BFC041E12D0A2230370019B47704380E3
:1084D000099B057146710C220830002B07D019004A
:1084E00003F0E2FB2100009803F06EF9F7BD099953
:1084F00003F022FBF6E737B5041E0FD04388002BAC
:108500000CD00025C1881323007A1722019500950D
:10851000FFF7CDFFFF2365806372257037BD000034
:1085200010B50C4904004A88002A09D08B89002B19
:1085300005D00020CB8A0222834201D010BD012247
:1085400013000A20434300204032C854C818428018
:108550000472F3E71A65FF1F00234380037070471E
:10856000094B00211A0010B55C88002C06D01C793C
:10857000844203D10A234B43D01810BD01310A3382
:108580000329F1D10020F8E71A65FF1F10B5040098
:10859000407A03F049F9FF23637210BD704704303D
:1085A00010B580B203F038FB002803D00421494203
:1085B00003F0DAFA10BD000070B50025104CA06879
:1085C0002580A581A580A84202D003F085FAA56088
:1085D00000250C4C0C4B606D1D80230058331D7022
:1085E000A84202D003F078FA65650025606800288B
:1085F00001D003F071FA013508340A2DF6D170BDAF
:10860000E065FF1F8465FF1FD465FF1F70B5041E62
:1086100009D1054D2880A881A880A868002802D02B
:1086200003F05AFAAC6070BDE065FF1FF0B54B88EF
:1086300085B00193002343600A7905000F00022AE8
:1086400000D07BE0CA88032A17D98B685E78197836
:108650003602DC78D8790E4399781B7A24021B0203
:108660000C43034353495BBA0B80331D93421ED125
:10867000042C04D0631F022B0ED9012015E0019AAF
:108680004D4B1201D35A002B06D00198FFF7BEFFC5
:108690004A4A1369013313610421B8682E812C8082
:1086A000494203F061FA6860002005B0F0BD434D17
:1086B000042C06D0631F022B0FD9EB680133EB604B
:1086C000DBE7019A3C4B1201D35A002B05D00198ED
:1086D000FFF79CFF2B6901332B61374B300002936E
:1086E000019B029A1B010193002301998C468B5236
:1086F000130063449C8003939E81FFF750FF039B0C
:10870000041E986016D00421B868494203F02CFA80
:10871000FA880100043A200003F0C6FA0199029A8F
:10872000FB888A5A043B9B18029A8B522B680133B0
:108730002B60A2E7AB690133AB619EE71E4B02934E
:10874000019B1E01029BF35A002B2DD002998C191C
:10875000A068002828D0012A26D1FA889B189BB24D
:108760007352A189994217D39B1AC018B96803F0B4
:108770009BFA029BA289F35A934200D07DE7002224
:108780002B81A3882B80A3686B60029BF2520B4A5B
:1087900053680133536070E7084A9368013393606C
:1087A0000198FFF733FF68E7044A536901335361C7
:1087B000F6E7C0464A65FF1FE065FF1F5065FF1FD3
:1087C00070B5051E15D10B4C0B4B18802300583388
:1087D0001870606D002802D003F07EF965652500F1
:1087E00050356068002801D003F076F90834AC42B7
:1087F000F7D170BD8465FF1FD465FF1FF0B517006A
:10880000A12285B0920001934243394B06001B68B8
:108810000C009B18D933FF331D78FDF741FF04305E
:10882000854204DD3000FDF73BFF0430C5B2BD4298
:1088300007D33A0000213000019B03F0DDF805B0BA
:10884000F0BD2900380003F08FFA2300C6B2503380
:108850001E700393019B29006365380003F0A4F99F
:10886000CBB20293002B02D0039B01361E70002670
:108870002300503303931B78B34204D8606D002863
:1088800031D10020DBE7029A2800002A04D0013B06
:108890001000B34200D02800F700E719387003F049
:1088A0001BFA786000280ED03A78019903F0FCF9A1
:1088B000019A3B780136D3180E4A0193D369F6B278
:1088C0000133D361D4E7039B18706065A74205D1DB
:1088D000084A1320D36A0133D362B0E7606803F01B
:1088E000FBF80834F2E703F0F7F800236365C8E704
:1088F0003409FF1F5065FF1FF7B50D000700042165
:10890000686803F031F92B89040003702B891B0A76
:1089100043702B8883702B881B0AC3702E89022515
:108920000436F6B2F42E15D81B4B9F4214D10C20FE
:1089300003F042FA1135011E0CD0902303708E3BD8
:108940000371043B4380154B8460C680187802F0A5
:108950003BFF00252800FEBD5C237B43104AD31853
:108960000093583301931B78002B0FD10300320082
:1089700038000099FFF742FF019B05001B78002B90
:10898000E8D13800009902F0C7FFE3E7054A072560
:10899000536A01335362DDE7FEFF00004865FF1FA5
:1089A0008465FF1F5065FF1FF0B587B0009017204A
:1089B0000F0016000193FFF7F2FD1325041E19D0D6
:1089C0000C98031E02D00199201D9847030AE370FA
:1089D000052302AAA0700430908127700098667069
:1089E00003A993800494FFF787FF051E02D020009F
:1089F00003F072F8280007B0F0BD0000F0B587B0B2
:108A00001F000CAB1B780391059301210DAB0600F1
:108A10001C78049200F0D6F81425002821D02000FC
:108A2000FFF77EFD0135041E1BD01149059B0A7816
:108A300003700132D2B2131EC68001D101231A0085
:108A40000B7022713000049B03990097FFF7ACFF75
:108A5000051E09D1230021000648074A093303F007
:108A6000F3F8280007B0F0BD002363802370F8E717
:108A70004C65FF1FF784001130750000F8B5050044
:108A80000E00064C064F2368002B02D03100280050
:108A900098470434BC42F6D1F8BDC046F065FF1FCC
:108AA0000466FF1F0123064A5B42538000231371B3
:108AB0005362044A136053609360D360136170473C
:108AC0000466FF1FF065FF1F0200002310B5064972
:108AD0009C000859002801D1625010BD0133052BBC
:108AE000F6D11320F9E7C046F065FF1F034A53880B
:108AF000181A434258414042104070470466FF1F15
:108B0000F0B585B002930AAB1F780CAB1B880090C0
:108B100008000E0001920393FFF7E8FF0500112003
:108B2000002D1BD10E48FFF7E1FF04001520002C9B
:108B300014D006220B99A771E01D03F0B5F8019B34
:108B400030002371029B29006371009B66802370B3
:108B5000039B6562E381FFF791FF280005B0F0BD3C
:108B6000FFFF000010B5FFF7C1FF04000220002C3A
:108B700012D060880121FFF781FF606A002801D0D0
:108B800003F09AF828220021200002F0D5FF0123EB
:108B900000205B426380207110BD000030B5074AA1
:108BA000074C5588010013780020A54204D05B1AB9
:108BB00059424B415842104030BDC0460466FF1F29
:108BC000FFFF0000084A10B501230C00904208D0B6
:108BD000FFF78CFF031E04D0037923405A1E9341F4
:108BE000DBB2180010BDC046FEFF0000024B187932
:108BF000431E9841C0B270470466FF1F70B5040061
:108C00000D001600FFF772FF002804D10D4B9C42A7
:108C100000D0143070BD416A03790520002907D0C7
:108C200012221A40102A02D10520002EF2D10F2064
:108C3000DB06EFD5897E0C20A94289414942494291
:108C40000840E7E7FEFF0000030010B5002800D150
:108C500010BD0348034A41889142F9D09847F7E78D
:108C60000466FF1FFFFF0000002330B5C45CCD5C2D
:108C70006C40D4540133102BF8D130BD0F230022A7
:108C800010B5C45C64002243CA54C25CD209013BE3
:108C9000F7D210BD0200010010B52032103103F0F0
:108CA00043F810BDF0B58BB003901020059317006A
:108CB000049102F081FF0090102002F07DFF009BE4
:108CC00013240190002B05D000280CD11324009808
:108CD00002F0F2FF019B002B02D0180002F0ECFF23
:108CE00020000BB0F0BD102002F066FF060010203F
:108CF00002F062FF13240500002E00D1AEE0002830
:108D000019D01022002102F017FF32002900039829
:108D100003F00AF8041E0ED133787F2B51D83000AF
:108D20000099FFF7ABFF009B1B787F2B53D801996D
:108D30000098FFF7A3FF300002F0BEFF002D02D025
:108D4000280002F0B9FF002CC1D1102002F034FF3E
:108D50000600102002F030FF0290002E7CD0002888
:108D600078D03A000F3223000125121105D00F33BD
:108D70003B4015B25A4253411BB26A1E1201002BEE
:108D800033D0049BD2B298180099029AFFF76CFF77
:108D9000013D10220021300002F0CEFEADB2049F52
:108DA0002D017D19AF4242D0002C33D0300002F0AB
:108DB00083FF029B002B00D189E7180002F07CFFA3
:108DC00085E729003000FFF759FF28002549009A60
:108DD000FFF74AFFA7E729000098FFF74FFF280099
:108DE0002049019AFFF740FFA5E70F210F400499A2
:108DF0008A18D9B28F4208D9D15C06A81954013318
:108E0000102BF6D1029A0199C0E7791A48424141E4
:108E1000C901F2E73900300006AAFFF725FF32004A
:108E2000039806A902F080FF10370400BAE7002C6F
:108E3000BCD13000029906AAFFF716FF320006A93E
:108E4000039802F071FF082204003100059802F037
:108E50002BFFABE71324A9E71324AAE7002800D0CF
:108E60006EE733E734C00011F0B58BB00F00160089
:108E70000225009000283FD0002A3DD00B1DDBB218
:108E80001800029302F098FE1135041E34D0FDF74D
:108E900047FD05003A000099201D02F0E5FCEBB209
:108EA0000393E3702B0CDBB22F0A00936370FFB2C5
:108EB0002B0E2370A7700193FDF72CFD10220100EB
:108EC00006A802F0D1FC2100029A04AB06A8FFF725
:108ED000E9FE051E0DD1039B08223370009B04A9F7
:108EE000B370019B7770F370301D02F0BDFCFDF78D
:108EF0001DFD200002F0E0FE28000BB0F0BDF0B533
:108F00008FB00D00149E039004920593002A03D1A4
:108F1000022420000FB0F0BD002EF9D00398FFF717
:108F2000E5FD1424071EF4D07278337812021A4338
:108F3000B3781B041343F27812061A43036A0192B2
:108F4000934201D30133E3D1002D03D03B790124B7
:108F50009B07DED50822002106A802F0EDFD059B47
:108F600013240433DBB21800029302F025FE051E21
:108F7000CFD0059A0499043002F076FC0422310027
:108F8000280002F071FC3900102210310AA802F00A
:108F90006BFC2900029A06AB0AA8FFF783FE041EA9
:108FA0000FD1082206A908A802F05EFC0822311D94
:108FB00008A802F0E9FD012807D101990398FDF7FF
:108FC000C9FC280002F078FEA3E70124F9E70000BD
:108FD00070B51C4C05002368181E10D0002D14D14C
:108FE0001A78002A0CD1981C083202F05DFE02F0BB
:108FF0001BFE0135002808D123681D70012070BDBB
:109000000A331800082202F04FFE2368002BF5D027
:10901000122002F0D1FE061E0DD0C123216803707C
:10902000457002311022023002F03EFE236831000A
:10903000587802F0C9FB206802F03EFE002323604E
:10904000DCE7C0462C66FF1FF8B504002020FDF7C2
:1090500055FB0D4EA700BB590500002B0DD0002875
:109060000BD0D878FF2809D108492A000C55F359AC
:1090700007480333611802F0E7FDF8BD290002F04C
:109080003BFE0028F0D1F8E74866FF1F3066FF1F5F
:10909000A1A2001170B5064D84006359002B05D0C4
:1090A000D87802F0C1FBFF226359DA7070BDC04668
:1090B0004866FF1F70B506008CB00C00150000213B
:1090C0003022684602F038FD31001022684602F076
:1090D000CBFB1D2021000322684402F0C5FB68463B
:1090E000FFF7D8FD2D21040003222800694402F077
:1090F000BBFB20000CB070BDF0B50700160097B0A8
:1091000001931CAB1D7830221EAB00910AA80021F0
:109110001C7802F011FD102239000AA802F0A4FB0D
:109120001022002102A802F007FD0722310002A848
:1091300002F09AFB072202AB9818631E9C4101992A
:1091400002F092FB02AB9C732B005A1E934102AAC1
:10915000D3730021102206A802F0EEFC06221D990E
:1091600007A802F081FB1A2002ABC01806221F9943
:1091700002F07AFB102200990EA802F075FB102273
:1091800002AB0EA908781C78013A6040D2B2087090
:1091900001330131002AF5D10AA8FFF77BFD102227
:1091A00012A904000EA802F07FFD102206AB0EA942
:1091B00008781D78013A6840D2B208700133013155
:1091C000002AF5D10AA8FFF765FD04431022209874
:1091D000E4B212A902F048FB200017B0F0BD70B550
:1091E0000E0014008CB00100102268461D0002F031
:1091F0003BFB3100082204A802F036FB21000822C4
:1092000006A802F031FB6846FFF744FD0400102277
:10921000280008A902F028FB20000CB070BDF8B5AA
:1092200006000D0000243719AC4200D3F8BD02F04F
:109230007BFB030A3B70631CDBB201379D4203D901
:109240000234F054E4B2EEE71C00EDE773B506001B
:109250000C000225002819D0002917D0032101A8ED
:10926000FFF7DDFF6B469A793F231A400133134322
:109270006A463000937101A92200FFF71BFF051E0B
:1092800004D10322E01C01A902F00EFD280076BDE6
:1092900003785807DA08C00FD20080009B071043FC
:1092A0009B0F1843C0B2704707230B40C908C90081
:1092B0000B4303707047000070B50400FFF7EAFE2F
:1092C000134DA4006359002B21D0186A002801D047
:1092D00002F0F2FC2B59986E002801D002F0ECFC51
:1092E0002B59D86E002801D002F0E6FC2B59186FDC
:1092F000002801D002F0E0FC2B59586F002801D063
:1093000002F0DAFC285902F0D7FC00232B5170BD83
:109310004866FF1F0E4B8000C35870B50C00002B31
:109320000FD09D68002D0CD02B78201D0B706B7812
:109330004B70A97CFFF7B8FF2B7E23726B69E3604B
:1093400070BD10220021200002F0F6FBF8E7C046B5
:109350004866FF1F014B18607047C0464466FF1FF8
:10936000074A03008000825810B5002A06D0D08832
:10937000984203D1012901D1FFF79EFF10BDC046DD
:109380004866FF1FF0B5264E95B087000B93BB597A
:109390000500099112200A92002B31D0D888FFF7DE
:1093A000A5FB04001420002C2AD0280010A9FFF7E8
:1093B000B1FFBB591E781D6A002E23D00895FDF71A
:1093C000EFFA07000020FDF7F1FA0790A379E61DF8
:1093D000069310AD0CA9089800F0E2FA0EA9280037
:1093E00000F0D7FA0B9B0A990493069B0998029305
:1093F000079B0396019300970EAB0CAAFFF77CFE28
:1094000015B0F0BDFDF7CCFA06903000FDF7CEFAAE
:10941000E31DA779079310AB06000893DAE7C0466F
:109420004866FF1F30B50C4C85002A59030085B0F3
:109430000120002A0ED018006946FFF76BFF2B5958
:109440001A78D888054B002A00D1054B6A460721B7
:1094500000F0D9FB05B030BD4866FF1F939900119D
:10946000A199001130B5094C8500295985B0102209
:109470006846253102F018FC2A591121044BD08886
:109480006A4600F0C0FB05B030BDC0464866FF1F0D
:109490003D9A001130B5094C8500295985B010223C
:1094A0006846353102F000FC2A591121044BD0885E
:1094B0006A4600F0A8FB05B030BDC0464866FF1FF5
:1094C0007B9A0011F7B54D4F86001020F4590D001E
:1094D00002F072FBF3592062186A132200286CD044
:1094E000033A29009C6802F0DFFBF3591A780192D5
:1094F000002A58D11E6A227D317B944651400122B8
:10950000019F114201D167461740217D91433943A4
:109510002175377B4F40BC4660460027800701D449
:109520004F081740012102208F40227D82433A4399
:109530002275377B5740BC4660460027400701D460
:1095400097080F400420227DBF0082433A432275D2
:10955000627D002794466046727B42400A4201D1F8
:1095600067460F400121627D8A433A436275777BEB
:109570005740BC4660460027800701D457080F407B
:109580000220627D7F00824317436775767B00224D
:109590007E40760701D4BA080A400426617D920015
:1095A000B1430A4362756A78002A08D06278002ABB
:1095B00005D005220533DA7700221000FEBD042213
:1095C0002979114205D1A17C114202D10533033A18
:1095D000F1E7019A21782C78002A02D10A002100B3
:1095E000140018220429E8D8042CE6D8052060438A
:1095F000034A05331218525CDDE7C0464866FF1F78
:1096000044C0001110B50A001121024B00F0FBFA12
:1096100010BDC046D79A00110B0030B587B001AD20
:109620002B806B4604001100981D082202F03CFBC1
:109630002A000B212000024B00F0E5FA07B030BDF4
:10964000FF9A001110B50A001121024B00F0DBFA5D
:1096500010BDC046539B001113B50B0011006A46A4
:1096600013706B4604000622581C02F01DFB6A466C
:1096700008212000014B00F0C6FA13BD739B0011B6
:1096800010B50A001121024B00F0BDFA10BDC04612
:10969000C39B00117FB505000B4BAA00D4580800EE
:1096A000002C0FD0666F237FE28821780396266F07
:1096B0000296E66E0196A46E0094FDF709FC280060
:1096C000FFF7FAFD7FBDC0464866FF1F10B51721A2
:1096D000FFF7E0FF10BD000070B50A000D00064B5B
:1096E0000221040000F08FFA060029782000FFF71D
:1096F000D1FF300070BDC046A39A001170B586B08E
:1097000000236A461370836804001D78681E0A28C7
:1097100059D801A902F0A8FA060633373B3F434760
:109720004B4F5300180000F042F9062312284BD08B
:1097300000281BD16088FFF7D9F90823002813D02F
:109740004279002A47D1264B1A78072312070BD5F6
:10975000244B1A680723002A06D01668002E03D06F
:10976000290001AAB04703006A4613706B461B78B4
:109770006088002B2AD1FFF767FC06B070BD180087
:1097800000F06CF9D4E7180000F087F9D0E7180072
:1097900000F093F9CCE7180000F0ADF9C8E7180025
:1097A00000F0C3F9C4E7180000F0F6F9C0E71800AC
:1097B00000F0F6F9BCE7180000F013FAB8E718005B
:1097C00000F013FAB4E707236A461370694660880D
:1097D000FFF782FFD1E70523012AC5D1024BB8E785
:1097E000D564FF1F4066FF1F4466FF1FF8B52C4F6E
:1097F0008600F35904000D00002B40D0DA88824225
:109800003DD15A78062A33D11A78002A2ED0012069
:1098100099681A6A097D014206D0157B054203D07A
:1098200007225A700120F8BD0220014204D0157BA6
:10983000054201D00922F4E70420014204D0127B42
:10984000024201D00B22ECE7164B1B68002BE9D03B
:109850005B68002BE6D020009847BB5900215B785D
:10986000122BDFD12000FFF715FFDBE70E4BECE7F3
:10987000112A04D1002900D032252900F2E7002D59
:1098800008D12000FFF732F9002803D01023027915
:109890001343037121002800FDF798FAC2E7C04680
:1098A0004866FF1F4066FF1F4466FF1F70B50E4EDF
:1098B0008500AB590400002B13D01B78002B11D16D
:1098C0000A4B1B68002B04D05B68002B01D02000E2
:1098D000984773595B78122B03D100212000FFF7C2
:1098E000D9FE70BD024BECE74866FF1F4466FF1FC0
:1098F0004066FF1F094B8000C3581020002B0CD07E
:109900001A6A002A09D09B68002B06D0127A1B7EA7
:10991000101C9A4200D9181CC0B270474866FF1F3D
:1099200070B503000D0014000220002A30D0002979
:109930002ED013700B78081D53704B789370FFF77F
:10994000A7FCE070012002212B7A23716B7B03407E
:1099500063716A7B0A401343042263716E7B164075
:10996000334363716E7BF608F600334363712B7BE0
:109970000340A371287B014000200B43A371297B86
:109980000A401343A3712A7BD208D2001343A37168
:1099900070BD10B50A0001000120FFF7C1FF10BD26
:1099A00010B50A0001000220FFF7BAFF10BD70B524
:1099B00006000C000220002E30D000292ED0737833
:1099C000201D0B70B3784B70F178FFF76DFC01220E
:1099D0003579257271794B1008001340934010407F
:1099E0000343881010408000C9080343C9000B439B
:1099F0006373B1794B100800134093401040034348
:109A0000881002409200C9081343C9000B4321206B
:109A10002373FCF773FE854201D2122070BD222011
:109A2000257AFCF76BFE8542F7D823781820042BA3
:109A3000F4D86378012BF1D80020EFE7030010B5CC
:109A40000220002909D0002B07D00322481C0A70ED
:109A500019000D3202F028F9002010BD0300022287
:109A6000080010B5002B06D0002904D00E32591C76
:109A700002F01AF90022100010BD030010B50220F8
:109A8000002909D0002B07D00422481C0A701900B5
:109A90000C3202F009F9002010BD10B5FFF7DEFF0F
:109AA00010BD03000220002906D0002B04D005229F
:109AB00000200A701B784B70704703000220002BB7
:109AC00008D0002906D05B7800200B70013B082BE2
:109AD00000D918307047030010B50220002909D0C2
:109AE000002B07D00622481C0A7019000A3202F027
:109AF000DBF8002010BD10B5FFF7B0FF10BD02006D
:109B00000B00022010B500290ED0002A0CD007212E
:109B10001970118859701188090A99701118082252
:109B2000D81C02F0C1F8002010BD03000A0002207A
:109B300010B5002B0CD000290AD09978587809026A
:109B400001431180901CD91C082202F0ADF80020BE
:109B500010BD030010B50220002909D0002B07D04A
:109B60000822481C0A701900921802F09DF8002083
:109B700010BD02000B00022010B500290BD0002AF6
:109B800009D009211970117818185970511C062232
:109B900002F08AF8002010BD10B5FFF75FFF10BD7E
:109BA00002000B00022010B5002A09D0002907D0BE
:109BB0005178197011180622581C02F075F800200F
:109BC00010BD030010B50220002909D0002B07D0DA
:109BD0000A22481C0A701900063202F065F80020BB
:109BE00010BD10B5FFF73AFF10BD02000B000220B8
:109BF00010B5002A06D0002904D018005178FFF7CC
:109C000053FB002010BDF0B585B017001E006A465A
:109C100006230500080091819380FEF7C0FC132401
:109C2000011E02900CD03800B047041E05D1280058
:109C300001A9FEF76FFA041E02D0029801F04CFF52
:109C40002800FFF701FA200005B0F0BDF0B50400D0
:109C50008BB0019115000021102202A801F06CFFC9
:109C6000334EA700B85900283CD0C388A34239D14D
:109C70000378002B36D14278062A18D10200010061
:109C8000553235310C3006ABFFF7A9FA002829D13F
:109C90002000FFF72FFE020006A902A802F004F838
:109CA000200002A901F080FE01200BB0F0BD816E02
:109CB000002917D00B8A112A28D19D420ED1019874
:109CC0001231093A01F060FF012807D1BB59200089
:109CD0009D6EFFF70FFE29000200DEE73221200013
:109CE000FFF7D8FC2000FEF701FF061E1BD0416ADB
:109CF000002918D00B8AAB4215D1082201981231E5
:109D000001F042FF01280ED1716A0AE09D42E9D1BB
:109D100008220198123101F037FF0128E2D1BB5926
:109D2000996E8A7EB9E7200001F046FDBCE7C04687
:109D30004866FF1FF0B56B4D87007E5985B03378BC
:109D400002900393002B00D087E0B368346A01933C
:109D50007078062817D101221B7D134202D0217B87
:109D6000114218D10222134202D0217B114251D15B
:109D70000422134203D0237B134200D08BE0019BCB
:109D80005A7DEB5991E007380428F8D801F06CFFB0
:109D9000032E42678300B36E002B03D11C2001F019
:109DA0000BFFB066EB599C6E002C1CD010220021DA
:109DB000200001F0C1FE0298FFF79CFD0100200089
:109DC000FFF72DFA01F0B0FD2082200008211230AB
:109DD000FFF725FA0298FFF78DFDA076EB592100D9
:109DE000D888FFF70FFC0822EB591CE0B36E002B5C
:109DF00005D01A00198AF0881232FFF70DFC0222F2
:109E0000019B197DEB5911423DD0207B10423AD085
:109E1000073208E0F488FCF7DBFD01002000FFF7C3
:109E200011FC0A22EB595A70029B9C002A59537864
:109E3000073B042B11D8D088FEF758FE00284ED0DF
:109E4000C3895A08D2182849029B0298CB542B592F
:109E500041180433254801F0F7FE05B0F0BDFCF7CA
:109E60009FFD03000120834201D100200393EB59A1
:109E7000DE88FCF79BFD039902003000FFF7ECFB46
:109E8000019AEB59117D042211420CD0217B114221
:109E900009D00B22C7E7F688FCF73CFD0100300033
:109EA000FFF7EEFB6BE7019A527D01210A4204D0D5
:109EB000607B084201D00C22B5E702210A4204D09F
:109EC000607B084201D00E22ADE704210A4204D093
:109ED000627B0A4201D01022A5E71222A3E7FA22F0
:109EE0005200B0E74866FF1F4C66FF1FABA200118F
:109EF00010B5064B1A780423100018401A4200D0FF
:109F00000348FFF727FA002010BDC046D564FF1FA5
:109F10008843FF1F70B50400FFF7D4FA051E43D134
:109F20002000FFF77FFA234EA400A0598268937C9B
:109F3000DB0708D50321036A1B790B40012B02D1F3
:109F4000017F0B430377431DD97F8B1E022B0DD856
:109F5000022900D00121C088FCF790FF0421335969
:109F60001A7F59700A431A77280070BD01290CD155
:109F700002231022437000210C3001F0DDFD305926
:109F800010213530FFF74BF9EEE70529ECD102231C
:109F9000D118437010220C3001F086FE0423325990
:109FA000117F0B431377EAE708251828DCD1053D1C
:109FB000DAE7C0464866FF1FF0B58BB005914388CD
:109FC0007E4F9E00F45915000493002C15D10129F1
:109FD00002D000200BB0F0BD101D57781678FFF7A7
:109FE00057F9EB68320002932B7A049901930090A1
:109FF0003B002000FCF70CFFEBE7E388049A934258
:10A0000001D00820E6E72378012B00D1D4E0059B9E
:10A01000581E092800D9CFE001F026FE05CE0A29F6
:10A02000CC506C859AB229000498FFF773FFD1E7F2
:10A03000200029001022453001F036FEB9594B7836
:10A04000042B02D1013B4B70C3E70B000A00253300
:10A0500035320C310498FFF795F90498FFF702FAAE
:10A060000522431E9841BB59C0005A70B2E7200038
:10A0700029001022553001F017FE049B4F4C9D0023
:10A08000295904980A0006AB55320C31FFF77AF9CA
:10A0900029591022453106A801F076FD012808D182
:10A0A0000498FFF7F7F90590002804D106222B59F0
:10A0B0005A7005988EE708230593FAE763780C2B0E
:10A0C0007AD1E36E002B03D11C2001F075FDE06610
:10A0D000BB59D86E00286FD01022290001F0E4FD92
:10A0E000BB590498DC6EFFF705FC0D22A076BB5926
:10A0F0005A706EE7E06E00285ED063780D2B5BD15E
:10A100002B8808220382A91C123001F0CDFDBB5917
:10A110009A68517D0222114226D0186A407B104273
:10A1200022D00C32E4E763780E2B45D1236F002B4D
:10A1300003D1162001F040FD2067BB59186F00289D
:10A1400003D01022290001F0AFFD0F22BB59CFE749
:10A1500063780F2B30D1206F0622691C103001F07C
:10A16000A3FDBB599A68517D0422114203D0196A9C
:10A17000497B1142D5D100210498FFF78BFA28E7DB
:10A18000636F002B0DD0BB59586F0028F3D01022FD
:10A19000290001F089FD0122BB5952425B6F1A610F
:10A1A000E9E7142001F008FDBB5960675B6F002BE5
:10A1B000E9D126E72978DFE707200BE74866FF1F8C
:10A1C00010B5064C207001F0E7FB06212078FDF762
:10A1D00091FF0348FEF778FC10BDC0465B66FF1F89
:10A1E0006193001100200BB270B50D00834216DAA6
:10A1F000264B187801F058FC041E0DD00378922BE2
:10A200000ED0A02B37D0224B1878FF283AD021004F
:10A2100001F0DAFA002835D180200002684070BDD4
:10A2200043780E2B0BD03E2BEDD18378052B12D02B
:10A23000082BE8D181798088FFF7D8FA08E0154B20
:10A2400082889A42DFD183681878591CFEF7C0FED5
:10A25000002817D1D7E7104B1B785B0712D50F4B9F
:10A260001B68002B0ED09B68002B0BD0C289811D70
:10A2700080889847ECE7FFF741FAA068002801D0F2
:10A2800001F02AFC200001F0A7FAC5E75B66FF1F7A
:10A290008143FF1F18200000D564FF1F4466FF1F85
:10A2A00010B50078FFF712FA10BD10B50078FFF76F
:10A2B000FDFA10BD0C234343084A10B59B185A6899
:10A2C000002A03D0012901D1904710BD9B68002BC3
:10A2D000FBD00029F9D19847F7E7C0467866FF1F01
:10A2E00001238340094A10B5946B1C439463506B5F
:10A2F00098435063D46B20009843012901D120007A
:10A300001843D063116B0B43136310BD00800040F2
:10A31000F0B500240127154B85B0DA6B144E03927B
:10A320001A6C0192DA64019BE3403B4217D0039D13
:10A33000E5403D400295E5B202992800FFF7BAFFDB
:10A34000316A736A002908D03900002B01D00299C4
:10A3500079402800FFF7C4FF01E0002BF9D1013458
:10A360000C36172CDFD105B0F0BDC0460080004090
:10A370005C66FF1F064B01215A68C2400A4204D0A6
:10A380001B68C3401800084070471B6DF9E7C046C2
:10A39000008000400122064B8240002903D0D9688A
:10A3A0000A43DA607047D9689143D960FAE7C0463A
:10A3B0000038004030B5032444430F4BE25C1B19C6
:10A3C0009C785D7801232D1B0135AB40013BA340F8
:10A3D000A140DB430C00122807D80849920052180C
:10A3E000116819402143116030BD054A11680B40C6
:10A3F00023431360F8E7C0468BC0001108F000400B
:10A4000014F00040C21F70B5D4B20623092C0BD83B
:10A410000125084C9540002908D00021FFF7CAFF0C
:10A4200023682B4323600023180070BD2368AB43CF
:10A43000F8E7C04600380040214BF0B51B185B78A8
:10A44000022B21D1032444431E4A1F4EA35C121940
:10A450009478012215008540B76B013CE4B23D437E
:10A46000A240B563194C122815D89B0000290CD1C5
:10A4700017495B1899680A439A600123205C154AC2
:10A48000834011680B431360F0BD11495B18996854
:10A4900091439960F1E70E4B00290DD159690A43A8
:10A4A0005A61225C1328E8D00123203A93400A49DC
:10A4B000086803430B60E7E7596991435961F0E786
:10A4C0005C66FF1F8BC0001100800040D0C00011EF
:10A4D00000F00040A0F00040A4F00040F8B50024D7
:10A4E0001B4E1C4D1C4B1B5D012B1FD1194A926941
:10A4F000E2401A420BD00122B25693402200143A95
:10A50000D2B2022A09D815494A6913434B61013472
:10A5100002360C35172CE5D1F8BD0022B2560F4992
:10A520009200521891680B439360F0E7022BEED132
:10A53000E7B23800FFF71EFF01235840C1B23800D0
:10A54000FFF77AFF3800FFF715FF6877DFE7C046AF
:10A550005DC000115C66FF1F5D66FF1F00F00040DC
:10A56000012202388240054B002903D059690A4371
:10A570005A617047596991435961FAE700380040C0
:10A58000F8B50E0001210F008740114A0400D3687E
:10A59000FD43BB43D360831E8B4201D8FFF7E0FF2E
:10A5A00000212000FFF72EFF0A4A0B4B5168012EB5
:10A5B00005D139431B1951605E700020F8BD294058
:10A5C000516002221C1962709A6915409D61F4E77E
:10A5D00000380040008000405C66FF1F012210B57B
:10A5E0008240074B002906D019680A431A600121EE
:10A5F000FFF7C6FF10BD196891431960F7E7C04621
:10A60000008000400C2370B5002543430A4A29000E
:10A610009B181D70094B04001B185D70FFF7B0FFFD
:10A620000123A340064928000A681A430A60054925
:10A630000A689A430A6070BD7866FF1F5C66FF1F58
:10A64000348000403080004070B504000E00FF28C8
:10A6500013D003250540FFF7D5FF084AA3089B0048
:10A660009B183F22ED00AA40AE401968200091439C
:10A67000314319600121FFF78DFE70BD183800408D
:10A68000F8B50C244443134B0500E4186368002B11
:10A6900003D1A3681220002B1AD0022201270E4BEF
:10A6A00000215B195A7028002770FFF769FF636863
:10A6B0001E1E08D0A3683E00002B04D02800FFF720
:10A6C00059FE4640F6B228003100FFF709FE00208F
:10A6D000F8BDC0467866FF1F5C66FF1FF7B5C42053
:10A6E000FF222B4B80001958002491433F3A0A4324
:10A6F0001A508022274F5202274E1A60274B1D5DA9
:10A70000002D21D0A31E012B03D80121E0B2FFF7B9
:10A7100027FF012D18D11F4B9B69E3402B4213D01B
:10A72000E3B218000193FFF725FE01000198FFF73F
:10A7300055FFE3B2143B022B1DD801217156184A74
:10A740008D405369AB4353613B7F002B0DD0E5B285
:10A750002800FFF795FF2800FFF70CFE7B7F010024
:10A76000834202D02800FFF7A5FD01340C370236E2
:10A77000172CC3D1F7BD012100237156F3568D402C
:10A78000074A9B009B189A68AA439A60DCE7C04678
:10A7900000E100E05C66FF1F5DC000115D66FF1F09
:10A7A00000F0004010B501210400FFF7E9FE01238D
:10A7B000044A002011194B70A34091690B43936127
:10A7C00010BDC0465C66FF1F70B50E00150004008A
:10A7D000FFF718FF0C236343094A20009B189D6074
:10A7E0005E60FFF74DFFF021064B074A8900051E0A
:10A7F0005A5002D02000FFF705FF280070BDC04668
:10A800007866FF1F0000FF1F11A3001170B5134DE4
:10A8100007202C78002C1FD19822210052002800FC
:10A8200001F062F80123C420FF222B700C4B800042
:10A830001C635C630B4B1C605C600B4B19589143B1
:10A840003F3A0A431A50802252021A600D20074AEA
:10A85000074900F0D9FF200070BDC0465C66FF1FAD
:10A8600000800040A0F0004000E100E0DDA6001103
:10A87000DDA40011030010B50620072B09D8054AF6
:10A88000137000F0C9FFD7210020034B034A890051
:10A890005A5010BDB043FF1F0000FF1FC91BFF1F10
:10A8A00070B51D0002240C2910D8094ACA40D207ED
:10A8B0000CD5FBF72FFF041E08D1059A0499280038
:10A8C000FBF744FFFCF7B2FDFFF712FB200070BD61
:10A8D0001210000030B50D7802232C009C43184262
:10A8E00001D02B431C0008252300AB43284201D094
:10A8F0002B00234320241D00A543204201D01C43EC
:10A9000025002A230D70184204D011781E3B0B43FA
:10A91000137030BD0028FCD10C2113788B43F7E76E
:10A92000F8B51D0006AB1B88140007AA0E000B200B
:10A930001778002B27D10A78022A49D14A68507823
:10A9400011780002244A08438018042840D801F0F6
:10A950008BF903121D1B2300F06801F01DF9021C86
:10A96000C0B2B84200D93A1CD2B22000F1682A80A5
:10A9700001F09AF906E00222F3681B882A8023700E
:10A980001B0A63700020F8BD0622EEE701232B802E
:10A99000F3681B782370F5E7F368002B16D00822C4
:10A9A0002A801A8822701A88120A62705A88A27045
:10A9B0005A88120AE2709A8822719A88120A627181
:10A9C000DA88A271DB881B0AE371DBE72B80D9E709
:10A9D00001202B80D7E7C04600D6FFFFF7B5160051
:10A9E0000A781D0008AB1F880C000123022A18D129
:10A9F0004A685078117800022B4A084380180328CF
:10AA00000FD801F031F902254439E06801F0C4F8AB
:10AA1000C0B20723B84204D37B190193152B02DD82
:10AA20000D231800FEBDE0682A003100C01901F0B6
:10AA30003BF96B4600209B88E268D0541B4B1B6897
:10AA4000834203D01B68834200D098470023E8E785
:10AA50000B23002FE5D1022DE2D1737832781B024F
:10AA60001343E2681380114B1B68002BEED01B6868
:10AA7000002BEBD00120E8E70B23002FD1D1062DCE
:10AA8000CED12A003100E06801F00EF9DEE70B2399
:10AA9000002FC6D1012DC3D132787533012AC0D819
:10AAA000E3681A70D2E7C04600D6FFFF6868FF1F50
:10AAB00070B50C001500072837D801F0D5F804143C
:10AAC00036361B36242E182015290BD8184E162280
:10AAD0000021300001F030F822002900300001F0A0
:10AAE000E3F8002070BD18200229FBD11288114B19
:10AAF0001A80F6E718200829F4D10A000E48290028
:10AB000001F06AF9EDE718200129EBD10B4B107821
:10AB10000B49DA69FFF7DEFEE3E718200129E1D1EE
:10AB2000064B10780749DA6BF4E70220DAE7C046F3
:10AB30005068FF1F2E44FF1F2444FF1FB443FF1F14
:10AB4000DC43FF1FFC43FF1F030010B50020DB07A1
:10AB500004D50721024A034800F08CF810BDC04616
:10AB6000E8C00011B443FF1F054A03001068002825
:10AB700003D082889A4201D1806870470068F6E766
:10AB8000606AFF1F0A88030008009A4204D08A887E
:10AB900004309A4200D0002070470000F8B5F2223D
:10ABA00000230D4F0D4E79680500424333709942E2
:10ABB00000D07B600A4C0021200000F0BDFF002384
:10ABC0001A007C60AB4202D100203370F8BD013323
:10ABD0002280DBB2F234F5E7586BFF1F566BFF1F84
:10ABE000646AFF1F73B56B46019006006846150046
:10ABF0001980FCF74DFF041E11D1002D0FD076896E
:10AC0000002E11D00C2000F0D7FF00280ED0084AEB
:10AC10000460136886808560002B02D110602000DC
:10AC200076BD1A001B68F7E70224F8E71324F6E75D
:10AC3000606AFF1F012100220A4B10B549420A4CED
:10AC4000198099809A719A70084B207001201980A0
:10AC50005A60FFF7A3FF2078FCF778FF0448FDF760
:10AC600033FF10BD7068FF1F606BFF1F586BFF1F25
:10AC700021AD0011022310B5002802D0FFF7B2FF6A
:10AC80000300180010BD0000030010B50020DB0712
:10AC900004D50421024A0348FFF7A4FF10BDC046B3
:10ACA000FCC000113444FF1FF0B50E2687B003939B
:10ACB0000CAB1F8802ABF6180500080031000292A9
:10ACC000FDF768F804000120002C0FD03088FFF752
:10ACD0004BFF03000E20002B08D05E68002E05D02D
:10ACE00021002800039B029A0097B04707B0F0BDEF
:10ACF0000A4B10B5984207D10122002352420A8024
:10AD00008B708A808B7110BDFFF73CFF0028FAD052
:10AD100001235B42038000238370F4E7FFFF000000
:10AD2000F8B5050001290AD1134E00243388F22713
:10AD3000AB4219D028001149FFF7DAFF06E00229DB
:10AD400004D10139FDF73EFF0028EDD0F8BD3B00EE
:10AD500063437268D018D35A002B09D03A000021FF
:10AD600000F0EAFE0134E4B2054B1B78A342EED8B2
:10AD700001235B423380DDE7586BFF1F7068FF1FC4
:10AD8000566BFF1F10B5FFF7FDFE03000020834246
:10AD900000D0987810BD0000F0B589B01C000EAB53
:10ADA00080CB03901E8810AB1B78049202930B7A21
:10ADB0000D00DB0616D42B780593022B24D00498C3
:10ADC000FFF7D2FE002812D003689C46002B0ED05D
:10ADD000029B2200019329003B00644603980096E1
:10ADE000A04705E00498FFF7BFFE002802D10E201F
:10ADF00009B0F0BD8368002BF9D00A22290003981E
:10AE000098470028D7D0F3E76B6858781A786B4BCF
:10AE1000000210439842D2D8043B984210D2684BAB
:10AE2000984242D015D8674BC0180128C7D80B20CC
:10AE3000002EDDD1EB681A7859683A80200028E0AE
:10AE4000614BC018032800D979E000F00DFF846A37
:10AE5000789E5E4B9842B2D10B20002EC8D10123C0
:10AE60003B80EB6831001B7823706889013080B229
:10AE7000FCF790FF3A88031E0ED0017802328A1840
:10AE80003A80428962704289120AA2705968027837
:10AE9000E01C00F009FF06E004323A803100042291
:10AEA000601C00F049FE0020A2E70B20002E9FD17D
:10AEB000EB6807A91E8804233B80330A3000267004
:10AEC0006370FCF767FF051E28D004AB9A890E2338
:10AED00004A95B183E49C668FCF7D0FF00280BD1D7
:10AEE0002B783C486A680599FBF786FB002803D15C
:10AEF000012304AA5B42D3813278022A06D1716809
:10AF0000201D00F0D1FE3B8802333B800E2304AAB3
:10AF10009B181B88A3701B0AE370C4E704ABDE8197
:10AF2000F4E70B20002E00D062E7E9680398FFF7F2
:10AF300029FF02233B802070000A6070B3E70B20DA
:10AF4000002E00D054E70222EB681B883A80237061
:10AF50001B0A6370A7E7E86800F01EFEC2B2030098
:10AF60000720B24200D243E70DD00299DBB271183C
:10AF7000994202DB921BD3B20293029BE9681A004A
:10AF80003B8089195AE70023F6E70B20002E00D0FA
:10AF90002EE70722EB683A801A7822705A7862709E
:10AFA0005A88A2705A88120AE2701A792271DA88D5
:10AFB0006271DB881B0AA37175E7C0460429000093
:10AFC0000228000000D8FFFFFFD6FFFF0328000083
:10AFD000FFFF00002CC00011F0B58DB06B460020C3
:10AFE000089120229B5E83423DDAA64B187800F040
:10AFF0005BFD071E32D00378B02B2CD100790238CC
:10B0000016281FD800F0E0FE17001E001E001E00CC
:10B0100031001E0096001E001D011E0052011E0080
:10B0200073011E00CD011E0050021E001E001E00F6
:10B030008E021E00E302944B94491B8878880B8093
:10B04000FBF71AF83800FCF79BFF914B1B68002BAD
:10B0500001D038009847380000F0BEFB8020089BE4
:10B060000002434018000DB0F0BDEE2200218748D9
:10B0700000F062FD0BAA3B7B7989388900923A0087
:10B080000D32FCF79FFD0400804B1B78002C3FD154
:10B0900046E0804B788805937F4B4100CB5A0BAE3E
:10B0A000073BDBB232880293002301937B4B2100E4
:10B0B00006930093059BFFF76FFE744D002810D197
:10B0C000069B3A8A1B889A420BD1380005991230A8
:10B0D00000F05AFD002804D02B7862899B00EB1801
:10B0E0005A80162306A81B18328820007989FCF79D
:10B0F000C5FE2B7804009A00AA1851880029C3D0F5
:10B100000133DBB22B70002807D006A9C98A9180D1
:10B11000634A12889A42BCD802E0012149429180D8
:10B12000002B04D059497888FAF7DAFF8AE73E897C
:10B130000A2479E000253E89574B06937B88069ABE
:10B140005B009B5A033B9D4202DB002DF0D05BE08D
:10B15000162206A812183B7B798900923A0030002B
:10B160000D32FCF72FFD0590002858D04689017A52
:10B170007888FCF7F1FC041E44D1464B788807938D
:10B18000069B4100C95A454B0439C9B206AAD28A66
:10B1900006930291019400930599079BFFF7FCFD2C
:10B1A000041E2FD1069B39491A88931C002D26D1E5
:10B1B0004B807988384B4900CB5A5119033B8B425D
:10B1C00020DD059B31485B8941190B71A91C0135B4
:10B1D000C9B2EDB2059145191B0A2B71059B2D498A
:10B1E0000433181800F060FD2C4B059A1B88D31807
:10B1F000DDB22C4B9E4205D00136B6B29CE74988A1
:10B200009942D6D0002D0CD0204C2800618800F047
:10B210001BFB207021007888FAF772FF12E7059C6B
:10B22000F0E7002C00D183E77B78142B00D109E7ED
:10B2300016493B794E800B700C717888FAF712FF33
:10B2400000E7162406ABE41821003889FCF7A2FDBC
:10B25000011E00D1B7E1788822880F4C45002C5B95
:10B260000A4D013CE4B2029400240F4B0194009576
:10B27000FFF792FD041E00D014E129007888FAF748
:10B280004FFFDFE6606BFF1F2043FF1F7868FF1F43
:10B290006C68FF1F6C69FF1FA864FF1F5C6AFF1FBB
:10B2A0001E43FF1FFFFF00007A68FF1F162406AB36
:10B2B000E41821003889FCF76DFD011E00D182E100
:10B2C00078882288AE4C45002C5BAE4D013CE4B240
:10B2D00002947C89AC4B01940095FFF75DFD041E40
:10B2E00000D0DFE029007888FAF724FFAAE60025DD
:10B2F000A44B1D803B00F6331B78A24A7888079246
:10B30000AB4208D99E4B12880693069943005B5ABC
:10B31000013B9A4203DB0799FAF716FF92E61624DF
:10B320006B00FB18059306ABE418059B21001889F8
:10B33000FCF730FD011E03D1059B01241E8973E734
:10B340007888924B2288069C099343001B5B904EA1
:10B35000013BDBB20293002300960193099BFFF7A8
:10B360001BFD041E02D0059B1E895DE77B88069AA3
:10B370005B009B5A079A108832881218934202DCAD
:10B380001B1A013B33807F4C023032880999001927
:10B3900000F08AFC2388328801359B182380EDB2A7
:10B3A000A8E70BAA3B7B7989388900923A000D32D5
:10B3B000FCF708FC00250590059B002B04D10A240E
:10B3C000002D00D16EE060E0059B7888197AFCF7CB
:10B3D000C3FB0100041E63D1694C6C4B7888069452
:10B3E0000993069B4400E45A694B063CE4B20BAE59
:10B3F000328807930294019100930599099BFFF706
:10B40000CBFC041E4CD1079B5E491B881A1D002DE6
:10B4100030D14A80059B5B4C5A8963191A716B1CA9
:10B420009BB2E318120A1A71162306A832881B1859
:10B4300079890598FCF722FDFF21AA1C2E1D0335F2
:10B440000B00059092B2B6B2ADB2002803D006ABA5
:10B45000DB8AD9B21B0AA218651911712B714C4DE8
:10B46000301D2A884949201800F01EFC2B88F61848
:10B47000B5B2A1E74988914207D17A88069952006E
:10B48000525AEB18053A9A42C4DC3E4C28006188B7
:10B4900000F06AFC207021007888FAF75FFED1E5A1
:10B4A000002DF2D13E89BFE6162606ABF618310014
:10B4B0003889FCF76FFC3D000400FA3500282DD0D8
:10B4C000037A9B060CD400227B8939897888009204
:10B4D0003A000C32FFF7E8FB041E10D03E8915E05D
:10B4E0003088FFF741FB00281AD08368002B17D063
:10B4F0002100122278889847041EE4D0EEE72B78CA
:10B50000002B02D17888FAF739FE00262B78002B21
:10B5100000D097E5002C00D194E585E60124DDE715
:10B520000E24DBE7162506ABED1829003889FCF759
:10B5300031FC041E47D0037A9B0611D4154A7B8840
:10B540001188994203D01448814207D11380134BCC
:10B55000F2261D780023D9B2A94221D30924A1E7FC
:10B560002888FFF701FB00282FD08368002B2CD000
:10B570002100122278889847041EDFD092E7C04647
:10B58000A864FF1F7868FF1F7A68FF1F6C69FF1FA0
:10B590005C6AFF1F586BFF1FFFFF0000566BFF1F09
:10B5A00031005943546801336018615A0029D2D1DF
:10B5B0003C0008342100F22200F076FB210078885C
:10B5C000FAF7E4FD3EE501246CE70E246AE71D4B23
:10B5D0001A887B889A4231D07888FAF7E1FD31E504
:10B5E000F223059851684343CD18C95A00291FD04A
:10B5F0003B7A012B0BD16C88AB887888AA1D00940C
:10B60000FFF752FB041E02D000233B722E88F22269
:10B610000021280000F090FA00232B80059B0133C5
:10B62000DBB20593084B05991B78064A8B42D7D8A5
:10B6300001235B421380002CCED0F5E500263400B8
:10B640000596EFE7586BFF1F566BFF1F70B50400A0
:10B650000E001500FFF796FA031E08D131000548C9
:10B66000FFF790FA03001120002B02D01C8000206D
:10B670009D7070BDFFFF0000F8B50B4F06003B78D2
:10B680000D001400FF2B0ED00A2000F095FB011EC8
:10B6900009D0B1230380002346800371C580048153
:10B6A000387800F091F8F8BD7544FF1FF7B50F002A
:10B6B00008A90600088809A90B240988002821D1B7
:10B6C0000234022B1ED1557813782D021D432B0016
:10B6D0008B4301937334002B14D1FB6830001900A5
:10B6E0000093FFF74FFB019C85420BD02A003000EE
:10B6F0000099FFF7ABFF041E04D12A0030007989BE
:10B70000FFF7BAFF2000FEBDF0B50E7885B00390BC
:10B710000AA805880120022E0DD14C68277864788C
:10B7200024023C43054FBC4205D10398DBB201968D
:10B730000095FFF7BBFF05B0F0BDC0460229000031
:10B74000034B10B51B68002B00D09847FEE7C0469E
:10B75000646BFF1F07B501A8FFF7F2FF044A054815
:10B760000021121A00F0C0F8F8F786F8FEE7C0468C
:10B77000686BFF1F7844FF1F01B40248844601BC78
:10B78000604700BF2933FF1F01B40248844601BC53
:10B79000604700BF9D36FF1F01B40248844601BCCC
:10B7A000604700BF8539FF1F01B40248844601BCD1
:10B7B000604700BF9136FF1F01B40248844601BCB8
:10B7C000604700BF091B000001B40248844601BC69
:10B7D000604700BF594F010001B40248844601BCD4
:10B7E000604700BF434D010001B40248844601BCDC
:10B7F000604700BFADAE000001B40248844601BC02
:10B80000604700BFF30E000001B40248844601BC4B
:10B81000604700BF4931FF1F01B40248844601BCA4
:10B82000604700BFC91BFF1F01B40248844601BC2A
:10B83000604700BF1147010001B40248844601BCC3
:10B84000604700BF0124000001B40248844601BCE7
:10B85000604700BF350E000001B40248844601BCB9
:10B86000604700BF8B52010001B40248844601BC0E
:10B87000604700BF4551010001B40248844601BC45
:10B88000604700BF2526000001B40248844601BC81
:10B89000604700BF5522000001B40248844601BC45
:10B8A000604700BFC539FF1F01B40248844601BC90
:10B8B000604700BF692EFF1F01B40248844601BCE7
:10B8C000604700BF9DA9000001B40248844601BC46
:10B8D000604700BFF94C010001B40248844601BC36
:10B8E000604700BF5934FF1F01B40248844601BCC1
:10B8F000604700BFB70E000001B40248844601BC97
:10B90000604700BF2124000001B40248844601BC06
:10B91000604700BF4538FF1F01B40248844601BCA0
:10B92000604700BF3119FF1F01B40248844601BCC3
:10B93000604700BF2951010001B40248844601BCA0
:10B94000604700BFF919FF1F01B40248844601BCDB
:10B95000604700BFE117000001B40248844601BC03
:10B96000604700BF5D17000001B40248844601BC77
:10B97000604700BFE932FF1F01B40248844601BCA2
:10B98000604700BF4550000001B40248844601BC36
:10B99000604700BF5952010001B40248844601BC0F
:10B9A000604700BFC926000001B40248844601BCBC
:10B9B000604700BF311B000001B40248844601BC4F
:10B9C000604700BFA930FF1F01B40248844601BC94
:10B9D000604700BF691F000001B40248844601BCF3
:10B9E000604700BF055E000001B40248844601BC08
:10B9F000604700BF6DBC000001B40248844601BC32
:10BA0000604700BF0519FF1F01B40248844601BC0E
:10BA1000604700BF851F000001B40248844601BC96
:10BA2000604700BF9137FF1F01B40248844601BC44
:10BA3000604700BFB352010001B40248844601BC14
:10BA4000604700BFED3AFF1F01B40248844601BCC5
:10BA5000604700BF3555000001B40248844601BC70
:10BA6000604700BF8552010001B40248844601BC12
:10BA7000604700BF6571010001B40248844601BC03
:10BA8000604700BF4D39FF1F01B40248844601BC26
:10BA9000604700BFC136FF1F01B40248844601BCA5
:10BAA000604700BF350E000001B40248844601BC67
:10BAB000604700BFF54E010001B40248844601BC56
:10BAC000604700BFED4A010001B40248844601BC52
:10BAD000604700BF413BFF1F01B40248844601BCE0
:10BAE000604700BFD949010001B40248844601BC47
:10BAF000604700BF2146010001B40248844601BCF2
:10BB0000604700BF713AFF1F01B40248844601BC80
:10BB1000604700BF0D52010001B40248844601BCD9
:10BB2000604700BF1D4B010001B40248844601BCC0
:10BB3000604700BFEDA5000001B40248844601BC87
:10BB4000604700BF154D010001B40248844601BCA6
:10BB5000604700BF291C000001B40248844601BCB4
:10BB6000604700BFC56D010001B40248844601BCB6
:10BB7000604700BF5549010001B40248844601BC3A
:10BB8000604700BFC130FF1F01B40248844601BCBA
:10BB9000604700BFCD4C010001B40248844601BC9F
:10BBA000604700BFDD52010001B40248844601BC79
:10BBB000604700BF090E000001B40248844601BC82
:10BBC000604700BF3D4B010001B40248844601BC00
:10BBD000604700BF193BFF1F01B40248844601BC07
:10BBE000604700BFC51D000001B40248844601BC87
:10BBF000604700BFB14E000001B40248844601BC5A
:10BC0000604700BF5125000001B40248844601BCD2
:10BC1000604700BF156B010001B40248844601BCB7
:10BC2000604700BFE928000001B40248844601BC17
:10BC3000604700BFD91B000001B40248844601BC24
:10BC4000604700BF5D3BFF1F01B40248844601BC52
:10BC5000604700BFA946010001B40248844601BC08
:10BC6000604700BFB54C010001B40248844601BCE6
:10BC7000604700BF713BFF1F01B40248844601BC0E
:10BC8000604700BFDD66010001B40248844601BC84
:10BC9000604700BF75A9000001B40248844601BC9A
:10BCA000604700BF056A000001B40248844601BC39
:10BCB000604700BFE94C010001B40248844601BC62
:10BCC000604700BF014C010001B40248844601BC3A
:10BCD000604700BF4D1F000001B40248844601BC0C
:10BCE000604700BF017F000001B40248844601BCE8
:10BCF000604700BF8D12000001B40248844601BCB9
:10BD0000604700BF5147010001B40248844601BCAE
:10BD1000604700BF053AFF1F01B40248844601BCDA
:10BD2000604700BF7918000001B40248844601BC96
:10BD3000604700BFE548000001B40248844601BCEA
:10BD4000604700BFC9A9000001B40248844601BC95
:10BD5000604700BF3D18000001B40248844601BCA2
:10BD6000604700BFA54F010001B40248844601BCF2
:10BD7000604700BF090E000001B40248844601BCC0
:10BD8000604700BF456B010001B40248844601BC16
:10BD9000604700BF3939FF1F01B40248844601BC27
:10BDA000604700BFC94A010001B40248844601BC93
:10BDB000604700BFC521000001B40248844601BCB1
:10BDC000604700BF1D4D010001B40248844601BC1C
:10BDD000604700BF853BFF1F01B40248844601BC99
:08BDE000604700BF810E000066
:10BDE800000101030200030304030502060207021F
:10BDF800080209020A030B030C020D000E030F03CD
:10BE0800100311001300140315001600493C00111B
:10BE18007D3C001100000000020000002ABE001155
:10BE2800192A0F180A000000F1590000FD2400002B
:10BE380041460100D1810011E5A1001139760011B8
:10BE4800D57F001165540011D9AF0011B150001110
:10BE5800593E0011893F001100000000161600002D
:10BE68000200000074BE0011F4FFF3FFD2FC0000D2
:10BE7800C9400011000000000000000054757961FD
:10BE88000042322E300030303139006769746875ED
:10BE9800622E636F6D2F7076767800544830354681
:10BEA8000000000002000000C0BE0011292A282A54
:10BEB800272A262A252A242A0A180000E204000034
:10BEC8007102000078EC00000500000074400000DA
:10BED8001027000060F00000040000000664000065
:10BEE800204E000000000000060000005C44000036
:10BEF800102700006CEE000007000000050000009D
:10BF08001F501D10023CB400000119002000000061
:10BF1800A1020000303132333435363738394142E6
:10BF2800434445460000000069580011BD580011FF
:10BF3800000000000200000048BF00116F2A6E2AAE
:10BF48001A18EAD8BC80F0FC60000000000000006D
:10BF5800000000F505D39727B6F615F7B777E6F092
:10BF6800C7F27200000001A0000000006410B71DB5
:10BF7800C8206E3BAC30D9269041DC76F4516B6B0F
:10BF88005861B24D3C7105502083B8ED44930FF0D1
:10BF9800E8A3D6D68CB361CBB0C2649BD4D2D38687
:10BFA80078E20AA01CF2BDBDFB349B5F80000080D4
:10BFB80000100000000000003B620011C57800116D
:10BFC8005F620011CD7C0011E3620011A37C0011B7
:10BFD80059630011797C0011AB630011417E001197
:10BFE80013640011417E001145640011FB7D0011AE
:10BFF80059630011317C0011D1630011D97D001102
:10C008000000000000000000B7640011D97D001195
:10C0180019650011DD780011052A042A012A002A71
:10C028000229032801280028011800180000000030
:10C03800000000000000000000000087010102016C
:10C0480002010102010203030401030101010101CC
:10C058000303020103000D000E001000110013007D
:10C068001401070108010A010B011C011D02040249
:10C0780005020702080219021A021C021D03010325
:10C08800020317000201000504000807000B0A005C
:10C098001716001D1C010201010504010E0D0111F6
:10C0A80010011413011716011A19020201020B0AD2
:10C0B800020E0D02111002141302171603050403D1
:10C0C8000807030B0A030E0D0001020307090A0BF8
:10C0D8000E0F101112141718191A1B1F20212200F5
:10C0E80021A90011DDA900110000000002000000D4
:10C0F80032C000110000000009B700110000000064
:08C108000200000030C000112C
:020000041FFFDC
:1000000000000000C13D001130BE00112CBE0011E7
:10001000A861FF1F000000000000000000000000B9
:1000200000000000000000000000000000000000D0
:1000300000000000000000000000000000000000C0
:1000400000000000000000000000000000000000B0
:1000500000000000000000000000000000000000A0
:100060000000000000000000000000000000000090
:100070000000000000000000000000000000000080
:100080000000000000000000000000000000000070
:100090000000000000000000000000000000000060
:1000A0000000000000000000000000000000000050
:1000B0000000000000000000000000000000000040
:1000C0000000000000000000000000000000000030
:1000D0000000000000000000000000000000000020
:1000E0000000000000000000000000000000000010
:1000F0000000000000000000000000000000000000
:1001000000000000000000000000000000000000EF
:1001100000000000000000000000000000000000DF
:1001200000000000000000000000000000000000CF
:1001300000000000000000000000000000000000BF
:1001400000000000000000000000000000000000AF
:10015000000000000000000000000000000000009F
:10016000000000000000000000000000000000008F
:10017000000000000000000000000000000000007F
:10018000000000000000000000000000000000006F
:100190004D33FF1F9531FF1FC166010000000000B5
:1001A000000000000000000000000000000000004F
:1001B000000000000000000000000000000000003F
:1001C000000000000000000000000000000000002F
:1001D000000000000000000000000000000000001F
:1001E000000000000000000000000000000000000F
:1001F00000000000000000000000000000000000FF
:1002000000000000000000000000000000000000EE
:1002100000000000000000000000000000000000DE
:1002200000000000000000000000000000000000CE
:1002300000000000000000000000000000000000BE
:1002400000000000000000000000000000000000AE
:10025000000000000000000000000000000000009E
:10026000000000000000000000000000000000008E
:10027000000000000000000000000000000000007E
:10028000000000000000000000000000000000006E
:10029000000000000000000000000000000000005E
:1002A000000000000000000000000000000000004E
:1002B000000000000000000000000000000000003E
:1002C000000000000000000000000000000000002E
:1002D000000000000000000000000000000000001E
:1002E000000000000000000000000000000000000E
:1002F00000000000000000000000000000000000FE
:1003000000000000000000000000000000000000ED
:1003100000000000000000000000000000000000DD
:1003200000000000000000000000000000000000CD
:1003300000000000000000000000000000000000BD
:1003400000000000000000000000000000000000AD
:10035000000000000000000000000000000000009D
:10036000000000000000000000000000000000008D
:1003700055B7001100000000000000000000000060
:10038000000000000000000000000000000000006D
:10039000000000000000000000000000000000005D
:1003A000000000000000000000000000491BFF1FCB
:1003B000000000000000000000000000000000003D
:1003C000000000000000000000000000000000002D
:1003D000000000000000000000000000000000001D
:1003E000000000000000000000000000000000000D
:1003F00000000000000000000000000000000000FD
:08183800706FFF1F4118FF1F34
:10184000024981F3088802F04FFB0000706FFF1F10
:1018500070B500241E491F4A1F484C6308CA1B0567
:101860001B0DE4188242F9D11C4B80228B630021AE
:1018700009201B4B920519621A4B1B4DDA671B4B53
:10188000DA688243DA609A68194802409A60112047
:10189000296002F0B7F8112002F094F880226B6CF6
:1018A000112093436B64EE23DB006343114A1B0C4E
:1018B00013840122104B9A7201F022FC0F4B1B780B
:1018C000002B04D10E4B1021187802F0FDFA70BDE8
:1018D000000005408805054000060540FF010000A6
:1018E00000F0004004E100E0003800403CF000401F
:1018F000FFDFFFFF7861FF1F2C62FF1F5A64FF1F8D
:101900005862FF1F10B502F04FF9072804D01228C3
:1019100008D0022808D010BD044A0420136B0133FC
:101920001363F8E70220F6E71420F4E75065FF1F81
:10193000F8B507000C0026002500503630785135E8
:10194000002804D10300287058342370F8BD29788A
:10195000CA00481E8141A3183800A25C5B68C9B266
:10196000FFF7D0FF00280DD12B78DA00A218013341
:1019700050602B703378044A013B3370136A013393
:101980001362D8E70123DFE75065FF1F5C23434361
:10199000074910B5C9180B0058331B78012B05D126
:1019A000FFF7C6FF034A936A0133936210BDC04636
:1019B0008465FF1F5065FF1F10B502F00DFA064A3F
:1019C0000121130010CB4942D967044B136002F088
:1019D0007BF9200010BDC04600E100E010001000BF
:1019E00010B5040002F0F8F9024B1C6002F06CF92B
:1019F00010BDC04600E100E010B5040002F0ECF9B3
:101A00004021094A200013688B43136000F0F6FA66
:101A100001F07EFC0022054B01201A60044B0432C9
:101A20001A6002F011FAFEE71CF00040C4F000401A
:101A3000C0F00040431E5A425341A022F0B5D201EB
:101A40005B421340154D164A40019B182A18127E1E
:101A50008BB00191002A1BD01A000832D46F0022EB
:101A6000E6B206AFE4B294420EDC2818C369002B3C
:101A700008D0019902AA117106AA049202AA16734B
:101A800003A898470BB0F0BD1978B9540132EAE7C2
:101A90001A7D1A7806AB01261A70E6E71068FF1F58
:101AA00000400040F0B5254B04004001C25C85B009
:101AB000002A2BD01A18117E002927D0917E0029E8
:101AC00024D01179022921D11689D788D168F51B34
:101AD000ADB22A1C102D00D9102292B2BE4217D1ED
:101AE0001818012303710023C269C38003819A423D
:101AF00006D06846032103730171029301A8904741
:101B00000820002C00D0192001F0FAFA05B0F0BD31
:101B1000013C65426C41A0256442ED012C40084D1A
:101B20001B186419074D0633013A92B2AA42EDD050
:101B30001888461C1E80085C2070F5E71068FF1F9F
:101B400000400040FFFF00000F220E4B10B59868C8
:101B5000104002380A280BD802F00AF80D0A0B0AC6
:101B60000A110A0A0A0A060002210020FFF762FF92
:101B700010BD0121F9E70020FFF794FFF8E7DB6FC4
:101B8000F6E7C046004000400F220E4B10B59868A3
:101B9000104002380A280BD801F0EAFF0E0A0B0A9F
:101BA0000A120A0A0A0A060002210120FFF742FF70
:101BB00010BD01210800F9E70120FFF773FFF7E7E7
:101BC000DB6FF5E70090004013B5334C2378072B0B
:101BD0003DD8324B1A78324B002A39D1802219680D
:101BE00052020A431A60252001F0CCFE20232D4A20
:101BF00011680B43802113606B460422C9050868F5
:101C00000733104228D080210422C905C868104239
:101C10002ED080212020C905CA688243CA601422C0
:101C20001A701A78002A2FD18021C905C86820327D
:101C30000243CA6014221A701A78002A28D11A4B5B
:101C40001A7D22785A601D221A705932DA6013BD4B
:101C50001A6816490A40C5E7086802430A60142258
:101C60001A701A78002ACED01A78013AD2B2F7E761
:101C7000C8680243CA6014221A7019784A1ED2B288
:101C80001A700029F9D1C4E71A78013AD2B2C7E72D
:101C90001A78013AD2B2CEE7B043FF1F7844FF1F53
:101CA0003CF00040A843FF1F00200040FFFFFEFF64
:101CB000564B70B51B68012B03D1554A936D013308
:101CC000936501F0C9FF534B534A1860534B544C72
:101CD0001A600123534A1360534A13602378002B80
:101CE00006D006225149524802F07EF900232370A3
:101CF000504A514B10681B78C1B2002B0ED14F4C8B
:101D0000C0B223785BB2002B4FDB237824785BB220
:101D100064B21B0424021B191B1813600B1C5029EE
:101D20004ED95023464A47491078DBB2FF22022899
:101D30004BD10868444C454D267890432A7896420A
:101D400054D9227824782E78023B5D10A31B6B4374
:101D50005201D31A10335B111843086002F024F9C2
:101D6000031F012B45D83A4B1B78002B06D0394B6B
:101D70001B78002B02D0002001F00EFFA122364B71
:101D800092009978354B4A431B689B188322920036
:101D90009B181B78033B012B03D8AF20400002F0B7
:101DA00003F801222E4BDA8270BD237824785BB2CF
:101DB00064B2FF33FF341B0424021B190138ABE764
:101DC000CAB2022AAED20223ACE70868254C264DDF
:101DD000267890432A78964208D9227824782D785C
:101DE000023B5B10641B63435201B2E72378DBB212
:101DF000B2E70228D5D11D4B1B78013B022B03D93A
:101E00001B4B1B78022BCCD16C20C8E79809FF1F15
:101E1000FC0FFF1F9C64FF1FFF3F000014100340D6
:101E2000A064FF1F0C10034000100340D50BFF1FE0
:101E30007211FF1FB40003408C09FF1F680AFF1FC7
:101E4000490AFF1F94000340460AFF1F470AFF1F6D
:101E5000F908FF1F2209FF1F300DFF1F3409FF1F64
:101E6000BC0BFF1F440AFF1F450AFF1F1C09FF1F71
:101E70002309FF1F10B502F03FF80022014B1A8022
:101E800010BDC0469A64FF1F10B501F0EDFFA121FF
:101E9000054A89009478054A61431268044B521838
:101EA000528C1A8010BDC046300DFF1F3409FF1F31
:101EB0009A64FF1F10B50D4B0D4A9978A1239B0022
:101EC0004B431268D218531DD97F0A4B1B88994285
:101ED00009D2441C07D0C82805D0D2695B1A5A43DE
:101EE000054B5343C01802F0B7F810BD300DFF1F6B
:101EF0003409FF1F9A64FF1F7102000070B5244D62
:101F00002B68002B28D002F00FF82B68D8402B68E4
:101F10000400002B27D001F0B7FF2B68D8401D4BE1
:101F20001D4A9978A1239B004B431268D118D25CBB
:101F300091239B00002A20D0CA580132CA50174B67
:101F400017491B680868834214D3D23B181A012A28
:101F50001AD0144B186070BD01F0E6FF124B1968DF
:101F600002F09AF8D3E701F08FFF0F4B196802F0E7
:101F700093F8D4E70D495B18E8E7CA500C4B1B688F
:101F8000DB68E418201AE4E7F530FF30E1E7C046EB
:101F90001C08FF1F300DFF1F3409FF1F9C09FF1F86
:101FA0009C64FF1FA009FF1F1808FF1F2DFF3F00A3
:101FB000A464FF1F70B504000D00282916D103008A
:101FC000A433C2881B889B1A0B4A9BB293420DD93B
:101FD00006006A3605223100653001F055FE002802
:101FE00004D13100200001F007FF70BD290020005E
:101FF00001F0CAFFF9E7C046FE7F0000F8B5050012
:10200000012001F089FE134CA36AA26A9342FBD11E
:10201000114E336001F0F8FE1049030008601048CB
:10202000426894460F4A17680022BC4501D24268B4
:10203000BA1A0D4802603268AD18A422E562606ADF
:10204000520302436262094A1278002A01D00F3B10
:102050000B60F8BD00F00040340AFF1FE408FF1FCA
:1020600028100040180AFF1F1C0AFF1F1C09FF1F31
:1020700070B580241025E405A3682B43A36001F00C
:102080001BFFA368AB43A36070BD0000F7B516004B
:1020900080221C001023D2050191916805000B439A
:1020A000936000225A4BD7301A6001F02DFE9D2319
:1020B0002A002F009B00EB58CA3201210092FC3706
:1020C000002B01D00021009A386801F0B5FD2900ED
:1020D000009BCB311A784F4BD3351A604B780A7876
:1020E0001B0213438A7812041A43CB781B0613434E
:1020F000494A1BBA13604B790A791B0213438A7948
:1021000012041A43CB7931001B061343434A1BBA0E
:1021100013606B782A781B021343AA7812041A43BF
:10212000EB781B0613433E4A1BBA1360019A330235
:1021300013433C4A13603C4B22001B1B9C46032963
:102140003DDCB3089A0013005142B21A032A46D16B
:10215000354AE018511A827840781204000202438E
:10216000E05C043302430A600022FF2B4BDDF022C7
:102170002E4B12011A600F222D4B1A602D4A136844
:10218000002BFCD00023224A27491360091B321D73
:102190000B191B68043A180A23706070180C1B0E88
:1021A000A070E3700434002AF2DC802210213B6826
:1021B000D20501333B6093688B439360F7BD634660
:1021C000D578981893782D061B042B43157804397D
:1021D0002B43557804322D022B430360AFE7022ACC
:1021E0000AD1114AE05C511AE218527812020243F5
:1021F0000A6004339BB2B7E7012AB5D10A4A521AE2
:10220000E15C1160F5E7084959180A600433ACE74E
:10221000000004403C000440380004403400044006
:10222000300004400C00044000010440040004405D
:102230001000044014000440F7B5150080221C0073
:102240001023D2050091916807000B43936000238F
:10225000654AD730136001F057FD9D233E009B0077
:10226000F9583B00CA363200FC33002900D07FE029
:10227000586801F0E1FC390032785C4BCB311A60D0
:102280004B780A781B0213438A78AC4612041A432F
:10229000CB78281D1B061343554A1BBA13604B7994
:1022A0000A791B0213438A7912041A43CB791B065D
:1022B0001343504A1BBA13604B7A0A7A1B0213432A
:1022C0008A7A12041A43CB7A21001B0613434A4A26
:1022D0001BBA1360009A2B021343484A1360220072
:1022E000474B1B1B0093009BCE785B1801938B78A8
:1022F00036061B0433430E78043833434E780431DA
:1023000036023343019E33600328ECDC0321A80826
:10231000431C9B002940800003292BD13849E51834
:102320005E18A9786D78E35C09042D0229431943EE
:102330003160030008330021FF2B2DDD314B324982
:1023400019600F21314B1960012327490B60304B75
:1023500019680029FCD006211B680B40042B20D0F3
:1023600080220020D20593680A318B439360FEBD22
:1023700001217DE7022908D121495D18E11849783A
:10238000E35C090219432960D3E70129D3D11C4931
:102390005918E35C0B60CCE7194818180160043346
:1023A000CAE7002310490B606346002B0CDC3B009E
:1023B000FC335A68102101325A608022D20593689A
:1023C00001208B439360D2E7009B9B181B68190A7E
:1023D00013705170190C1B0ED37004235B42917063
:1023E0009C440432E0E7C046000004403C00044046
:1023F0003800044034000440300004400C00044025
:102400000001044004000440080F000010000440D4
:102410001400044070B5061E19D002225A4B9B7955
:102420009343012B13D1594B1A78FF2A0FD15A78B5
:10243000FF2A0CD19A78FF2A09D1DA78FF2A06D12F
:102440001A79FF2A03D15B79FF2B00D199E0504B19
:102450000C201A78012A08D000224E4D1A702978D3
:102460000B00093B042B01D8212070BD4B1F012B11
:10247000FAD9454CA37B042B00D982E0A279032A28
:1024800000D97EE09A1ED2B2012A02D860881F28A5
:1024900077D9002E56D0012E73D1A0880128E3D021
:1024A000002907D1581E032803D801F061FB121739
:1024B00015122E702978481E032811D80025364B96
:1024C0001D602823237501F08FFCA84227D0A5802A
:1024D000CAE702212970EDE70421FBE70321F9E7B0
:1024E00007390129C0D82D490968C96A8906BBD5B1
:1024F0002B4908780028B7D1012A01D9002BB3D184
:1025000002230B708021274D2633890128782375FB
:1025100001F052FC80212878890101F0D5FC0123CB
:10252000A380214B1B78002B0AD0FA2280211F4B5D
:1025300092001B8809025A431A4B187801F004FCD8
:10254000002092E701F048FC2B78A680073B012B86
:1025500003D917482E7001F0EFFB114B114C1A787C
:10256000002A06D080210022207889011A7001F00B
:1025700023FC01F0A9FB80212078090201F01CFC5A
:10258000DEE7122071E7C046A60BFF1F6B09FF1F95
:102590001A09FF1F1C09FF1F4809FF1FA464FF1F22
:1025A0002309FF1F1B09FF1F2109FF1F2C09FF1F04
:1025B0000010004010B5002901D001F0CDFB10BD86
:1025C000F7B5604B01919978A1239B004B435E4A7C
:1025D000060014681022E418D6235B00E058362366
:1025E000FF33E35C00279343222B41D1574B0F3A33
:1025F0001A600760012501F027FD019B1880E82380
:102600005B00E35C002B01D0B34258DD0023504F48
:10261000FB70AD33FF33E3581A68002A03D09B8860
:10262000DB439B071DD03823FF33E35C002B18D01E
:102630009B235B00E35C002B13D1D133FF33E35CBE
:10264000B3420EDAA4235B00E15AE018090A023112
:1026500001F0E2FC23000122FE33013E01351A871E
:10266000FA70E8235B00E35C002B2AD0A8B2FEBD21
:1026700003683D00002BBED081880430090A023176
:1026800001F0CAFCD6235B00E3581F60B2E72300C9
:10269000B133BA00FF339858013781880430090AF2
:1026A000023101F0B9FCE8235B00E35CBB42EEDCE5
:1026B000E822F61AED1800235200A354A6E70027DB
:1026C000F1E7200001F0A8FB00281FD0002E1DDD3F
:1026D0007319882647190193B600200001F004FB06
:1026E0005A30800020184068013581880430090A7A
:1026F000023101F091FC200001F066FBA359013387
:10270000A351BD4202D0019B9D42E6D1114BE35C37
:10271000002BABD095239B00E35C002BA6D00E4B87
:10272000E15A0029A2D00D4AA35C994202D9013393
:10273000A3549BE700231A212000A35401F074FB4B
:1027400094E7C046300DFF1F3409FF1F00140340FB
:10275000E010FF1F5A020000720200005E0200003B
:102760000D4970B54A6E0D4CD2038B69D20BA24253
:1027700006D80B4D0224AA4204D901F06DFB70BDAE
:1027800002246442E21815007E2425402242F4D03F
:10279000A3432B438B61F0E700F000400A200000C8
:1027A000FC1C0000F8B51D4B1D4F1A78002A10D1F3
:1027B000BA7B002A02D101321A7003E0032AFAD050
:1027C000022AF8D001F010FB00220120154B1A70EC
:1027D000F8BD154B154D1C68154B9E7801232B70C9
:1027E0002878C0B200F09EFBBB7B002B0BD101F020
:1027F00053FBA1239B007343E41883239B00E4183D
:1028000023782B70E4E7032B02D101F0B5FAF0E74F
:102810000020022BDCD101F08FFBEAE71C09FF1F2F
:10282000A60BFF1F2309FF1F3409FF1F490AFF1FC3
:10283000300DFF1FF0B587B00EAD2F780FAD2D789E
:102840000593AC46634614000E4D0CAA12782E7800
:1028500003930D9B009201932200059B029701F0C8
:1028600053FB2E70012C01D0042C08D18022064984
:102870008B889343054A1278D20113438B8007B0AB
:10288000F0BDC0461C09FF1F6C11FF1F7809FF1F18
:102890000B001B3B70B504003020E02B0DD813005B
:1028A000E025493BFF3B9BB2ED00AB4205D8034B13
:1028B000200019825A8201F01FFA70BD8410FF1F98
:1028C00010B501F0C9F9054B00205B68052B04D950
:1028D000034A5268D20200D4980810BD001000408C
:1028E000FCE100E070B501F077FA0D4B1B68FC339A
:1028F000DC691D6AFFF7E4FF6419844204D2094BC6
:1029000001241B68002B07D004220024064B1A70F8
:10291000064A93690133936101F0D6F9200070BD36
:10292000A464FF1F9809FF1F2309FF1FFC0FFF1F4F
:1029300070B50C4D2B68FC335C6A01F04DFAFFF763
:10294000BFFF2B680025FC339B6AE318834204D247
:10295000054B1B68AB4200D1051B01F0B5F92800FF
:1029600070BDC046A464FF1F9809FF1FD722044B07
:1029700092009B5810B5002B00D0984710BDC04660
:102980000000FF1F10B501F0DBF8FFF7EFFF27494C
:10299000274BCA6D274C1A4084235B001343CB6539
:1029A000254B1B68186A01F0B7F9244B244A1A60BA
:1029B000244B254A1A60A022244B52001A60244B53
:1029C000187801F039FB2000224901F015F90023A5
:1029D000A3600233A360204B2049236003232048D7
:1029E000A36001F009F910221E4BFF201A6080221B
:1029F00052031A60802292031A60802212041A6025
:102A000001F0CAF8012001F09FFAFA20400001F01D
:102A1000C3F9582001F0C8F9134801F04DF901201D
:102A200001F00AFA072001F0FFF810BD00F00040A5
:102A300000FEFEFF14100040A464FF1F00000340CE
:102A40000180063DBC00034034080000A4000340A0
:102A50004A0AFF1F71020000C3090000FFFF3F0088
:102A60002810004000E100E030750000674E336838
:102A700088331B6883F3088801F0FEF9644A6549CE
:102A8000136800200B401360634B644A1B68934239
:102A900000D1A6E001F0A8F80221614A13688B4337
:102AA0001360FFF76FFF5F4B5F4C1878C0B201F007
:102AB000BBFA0023A3600233A3605C4B01202360B8
:102AC00001F02AF90323A36001F086F8040001F065
:102AD000C3F8050001F080F8554B186001F044FA86
:102AE000544B1968621A531EA14200D2130080226F
:102AF000D203934201D39B029B0A3268D16AC90771
:102B000000D471E04C491C0C09689BB24C435943FA
:102B10002402090A641803264849FC3293680A68AB
:102B200047489B1A474A0768126847499B18474A13
:102B30009A1833409208DB190A600360042B03D90A
:102B4000013233400A6003600E684149A619300023
:102B500001F0A2FA3F4F3E493B68C3183B6030008A
:102B6000019301F009FA3C4E30680818384930608A
:102B7000884205D9019B01333B6001F0FDF93160CA
:102B800001F072FA354B1B78002B0DD001F064F880
:102B9000334B621B196812188A4232D24919091B39
:102BA000091A304801F028F82F4E337A002B0ED046
:102BB00001F052F8621BF1681218914224D94919A8
:102BC000091B091A294801F017F800233372284B12
:102BD00083F3088801F020F8002001F005F801F0E7
:102BE000A3F801F001F85CE7DC0199000234641AF3
:102BF0005900641A09214B438033CB40A408E418E0
:102C000089E7FA218900CCE71A49DBE7A464FF1FB2
:102C10001CF00040FFFFC1FF0C0AFF1FB64121035B
:102C200010000040490AFF1F14100040C3090000B3
:102C3000100AFF1F340AFF1F380AFF1F200AFF1F58
:102C4000280AFF1F1C0AFF1F240AFF1FC4090000D7
:102C5000710200006008FF1F2C0AFF1F1C09FF1FE4
:102C6000E408FF1F00100040740BFF1F3C100040E1
:102C700000000020DC050000A022054B92009B58BC
:102C800010B5002B01D0984710BD01F00DF8FBE7FF
:102C90000000FF1FA122054B92009B5810B5002B8E
:102CA00001D0984710BD00F0FFFFFBE70000FF1FB9
:102CB000A222054B92009B5810B5002B01D09847DB
:102CC00010BD00F0F1FFFBE70000FF1FA322054B42
:102CD00092009B5810B5002B01D0984710BD00F012
:102CE000E3FFFBE70000FF1FA422054B92009B5867
:102CF00010B5002B01D0984710BD00F0D5FFFBE7C1
:102D00000000FF1F70B500F0A7FF4F4B186000F0E8
:102D1000C3FF0400C30702D401F0DEF870BD002237
:102D20004A4B1A604A4B18780138042829D800F019
:102D30001FFF0320181C2400200001F0EDF80128DB
:102D4000ECD0444C2378042B6ED101F0ADF8002870
:102D5000E4D001F001F9582001F026F80223237095
:102D6000DCE7200001F088F9E9E7200001F04CF9E8
:102D7000E5E7200001F010F9E1E7200000F044FF52
:102D8000DDE701F011F90500012808D1324B1B786D
:102D9000053B012B03D82000FFF76EFFD1E72D4B39
:102DA0001B78022B01D0052B20D1022D28D12B4BD3
:102DB0009B7BAB431CD12000FFF76CFF264B1878A0
:102DC0000128BED16405BCD4244925224B7B034293
:102DD00005D1233A13405A42534126331A000B7D42
:102DE0009342AED9322000F077FFAAE7022D07D137
:102DF000194B1B78052B11D12000FFF759FFDDE798
:102E0000012D0BD1012B03D12000FFF75FFF98E7C5
:102E1000062B03D12000FFF767FF92E7200000F0A8
:102E200043FF022D8DD1C9E7032B04D10C4B987CB5
:102E300001F02AF972E7072B00D06FE7094B987B66
:102E400001F0C2F86AE7C0469C09FF1F9809FF1FFE
:102E50009009FF1F2309FF1F1C09FF1FA60BFF1F5F
:102E6000BC0BFF1FD40BFF1FFA210A4B0A4A490073
:102E70001A640A4A5A500A4A04395A50094A08310F
:102E80009A64094A5A50094A5C315A50084ADA662B
:102E90007047C0460000FF1F3528FF1F3129FF1F64
:102EA000E528FF1F1524FF1FA527FF1FB51EFF1FC5
:102EB000891EFF1FF7B50B0CFF270122009300238B
:102EC0003C001E001D009446019089B262469A4063
:102ED0001000084018413618B6B2FF2F02D1012E5B
:102EE00000D19FB2009802401A41AD18ADB2FF2C3C
:102EF00002D1012D00D19CB20133102BE6D1032069
:102F0000012E07D1012D04D1019B2401E4191C706D
:102F10000138FEBD102EFCD10238102DF9D0023040
:102F2000F7E700008023F7B59C46264B264F019318
:102F30002649274A274D284C284B02281AD160469B
:102F400038600868264E30408026360330430860DB
:102F500001990978002909D11660224A2A60224A7B
:102F60002260E02219689143A03A1BE08021C90247
:102F70001160F2E766463E600F68194E3E408027BA
:102F8000FF023E430E600199097800290DD11760B8
:102F900001280ED1154A2A60154A2260E0221968DC
:102FA0009143C03A0A431A60F7BD8021890211603B
:102FB000EEE7E0210F4A02432A600F4A22601A68B6
:102FC0008A43F0E74B0AFF1FE0000340D8000340AC
:102FD00090000340000003405000034040000340C5
:102FE000FFFFE3FF0280063D804508220180063D89
:102FF000806608220080069880550822F8B51E4B8E
:1030000080261A68002014003440324232D11A68F7
:103010001A4F32431A6001223B68063093433B60EB
:1030200000F07AFE0122164D2B681E432E603B688D
:103030000A2613433B608027BF00124B1B683B42AC
:1030400011D1013EF6B2FF2E09D17E220E4B1C6833
:103050002B68E40B1440934323432B6005E00820C6
:1030600000F05AFEE9E7002EEFD180222B686008BD
:1030700093432B60F8BDC046C4F000405CF00040B4
:1030800018F0004068F0004060F0004010B500F01B
:10309000EBFD01215820034A00F09EFFFFF7AEFF31
:1030A00010BDC046600AFF1F10B5782200210348FA
:1030B00000F0CAFD00F0A0FF002010BD9867FF1FC0
:1030C00070B5040000F088FE00230C200B4A0100BC
:1030D00059438D18515C00290DD0A14208D101231C
:1030E00000246B7000F068FD00F0EEFD200070BD64
:1030F00001330A2BEBD11224F6E7C0469867FF1F75
:1031000070B5040000F068FE002319001D000D4A90
:103110001078002806D0A0420CD1557001310C3235
:103120000A29F5D1002B0AD100F066FF00F0CCFD92
:10313000002070BD5078461EB0411B18EEE700F02D
:103140003BFDF3E79867FF1FF7B504000C20002351
:1031500084460E4D019267465F43E85D7E19A042AA
:1031600012D000280BD10A4B9C4662461B780833CC
:103170001370019B70707C557160B360FEBD0133AC
:103180000A2BE8D10320F9E70720F7E79867FF1F2C
:103190009467FF1F8020F8B5484BC0051B68C12409
:1031A0008360474BFF251A68012313434361454B56
:1031B000A4001A68444B40211A60444B1A68444BDF
:1031C0001A60444B1A59AA431A51C52292009E58BC
:1031D000AE433143802699509F583F49F6010F4036
:1031E0003E439E509E5880273602360A3043985000
:1031F00080201A5900020A4002431A5104341A5915
:10320000364E3F04324080263A431A511A59360648
:103210001202120A32431A5108341A5980260A40FF
:1032200002431A51C32292009F58B446AF4337431A
:103230009F509F58294E0F4007439F509F5837403B
:1032400080263604374380269F509F5836063F021B
:103250003F0A37439F50C0221F59AF433A431A5188
:103260001A591202120A1643C6221E5192009C5885
:10327000AC4365462C439C509C5800250C40204391
:103280009850C72080001A58154C1140C0221202D5
:103290000A431A50134B1B78DB08AB4201DC0020B9
:1032A000F8BD2378002B06D0A368002B00D09847E8
:1032B00001350C34EEE71220F2E7C046AC43FF1FA5
:1032C000A843FF1FB0F000409067FF1FB4F000401C
:1032D0008C67FF1F00E100E0FF00FFFFFFFF00FF22
:1032E0009867FF1F9467FF1F030010B51F2809D8B8
:1032F000072200201340072404490A78A2431343FD
:103300000B7010BD00230620F5E7C0469467FF1F31
:10331000034A0449136800200B4013607047C046FD
:103320001CF00040FFFFC1FF054B06491B780A68EF
:1033300005485B0702401B0B134300200B607047DE
:103340009467FF1F1CF00040FFFFC1FF70B50C2504
:10335000FFF7EAFF0A4B1C780A4BE4086543ED18B7
:10336000002C01D1200070BD2B78002B06D06B689B
:10337000002B00D09847013C0C3DF1E71220F2E70A
:103380009467FF1F8C67FF1F1FB5002102220B00EF
:1033900001910091052000F017FC02230B490A68F7
:1033A0001A42FCD120230393039B5A1E0392002B45
:1033B000FAD1074A1368002BFCDA0B246C44200076
:1033C000012100F0F9FD207804B010BD90C8004044
:1033D00000C8004013B504000A4B0193019B002B69
:1033E00001D1112016BDFFF7CFFF23000340044297
:1033F00005D0052000F090FC019B013BEDE7180093
:10340000F0E7C046FFFFFF0707B500F0E5FC8022AC
:103410000821D205936A0191002B01D107399162ED
:1034200002210C4A11600199481E01900029FAD12D
:1034300003311160053101910199481E0190002965
:10344000FAD11160002B02D18022D205936200F0E4
:103450003BFC07BD00C00040F0B52D4C89B023787F
:10346000002B4FD1FEF7A8FA02232A4F03903A68A7
:103470001A42FCD120230693069B5A1E0692002B6B
:10348000FAD1254E3368002BFCDA0120FFF7A2FFAA
:10349000011E02D0112009B0F0BD030003220190EB
:1034A000009005AD9F2000F08FFB0321280000F065
:1034B00083FD02233A681A42FCD120230793079B1D
:1034C0005A1E0792002BFAD13368002BFCDA012038
:1034D000FFF780FF0028DDD10398FEF781FAAA7874
:1034E0006B7811041B020B4329780B4363601300B4
:1034F000113B0A49052B07D801239340A3600B60B9
:10350000012323700020C6E780231B03F6E7C04693
:103510009443FF1F90C8004000C800409808FF1F58
:103520001E4B30B55A6818781D4B85B0D3185942D8
:103530004B4101210093002300F016FC194B1A4A5D
:1035400002259A6300221A6510325A658022C4212E
:103550009D65164B1648D202DA6789004258154B12
:1035600080241A4080231B041343435064234120CA
:103570000393E40500F006FA402000F003FA6562C8
:10358000039D6B1E0393002DFAD103236362FFF7A3
:103590003BFFA562FFF760FF05B030BDA043FF1FF2
:1035A00095FFFEF700C80040050001FF04E100E0C0
:1035B00000E100E0FFFF00FFF0B585B00700FEF777
:1035C000FBF9022305002D4C22681A42FCD120236E
:1035D0000093009B5A1E0092002BFAD1284E3368AC
:1035E000002BFCDA0120FFF7F5FE002803D01124A0
:1035F000200005B0F0BD234B2360022322681A424D
:10360000FCD120230193019B5A1E0192002BFAD179
:103610003368002BFCDA0120FFF7DCFE0028E6D13E
:10362000194B1F60022322681A42FCD12023029307
:10363000029B5A1E0292002BFAD13368002BFCDA4F
:103640000120FFF7C7FE0028D1D1104B23600223D1
:1036500022681A42FCD120230393039B5A1E039233
:10366000002BFAD13368002BFCDA0120FFF7B2FE01
:10367000041EBCD12800FEF7B3F9B9E790C800409A
:1036800000C8004001000006A8C8004001800001F9
:1036900010B50020FFF790FF10BD000010B5064BDD
:1036A00018705960FFF73CFF00211320034AFFF711
:1036B0004BFD002010BDC046A043FF1F2135FF1F5A
:1036C000F0B5040085B003920291FEF775F98822E7
:1036D00063035B0B52051A438023DB059D6A80233D
:1036E000274F0092BA68002601901B039A420CD91A
:1036F000F82326001B041E401C4206D08022214BCA
:1037000052025E6219680A431A60002D0BD100F064
:1037100063FB02221C4B1A608023DB055A62013ACC
:103720009A6200F0D1FA0023039A934220D1002D2F
:103730000AD100F051FB144B03221D608023DB05EE
:103740005A629D6200F0C0FA8023BA681B039A4255
:1037500008D9002E06D000220A4B0C495A621A687A
:103760000A401A600198FEF73BF9002005B0F0BD51
:10377000009A0299D2181278CA540133D4E7C0468D
:103780009443FF1F00C8004000C00040FFFFFEFF41
:10379000F0B587B0029103920400FEF70DF9019095
:1037A00000F01AFB802302250122234EDB05356041
:1037B0005D629A6200F088FA204F3B682B42FCD190
:1037C00020230493049B5A1E0492002BFAD11C4D13
:1037D0002B68002BFCDA0120FFF7FCFD002802D04B
:1037E000112007B0F0BD2000039A029900F0CCFA36
:1037F000022304003A681A42FCD120230593059B5A
:103800005A1E0592002BFAD12B68002BFCDA0120FE
:10381000FFF7E0FD051EE3D100F0DEFA802303226E
:10382000DB0535605A629D6200F04EFA0198FEF7A2
:10383000D7F8E0B2D5E7C04600C0004090C80040CD
:1038400000C80040F0B5802489B00600FEF7B4F847
:10385000E405A36A02250393029000F0BDFA012358
:10386000304F3D606562A36200F02EFA2E4C236853
:103870002B42FCD120230593059B5A1E0592002B59
:10388000FAD12A4D2B68002BFCDA0120FFF7A2FDAC
:10389000002803D01124200009B0F0BD244B236080
:1038A000022322681A42FCD120230693069B5A1E4B
:1038B0000692002BFAD12B68002BFCDA0120FFF7CF
:1038C00089FD021EE6D11B4B03211E6003000190FF
:1038D0000090202000F078F9022322681A42FCD1DF
:1038E00020230793079B5A1E0792002BFAD12B68BF
:1038F000002BFCDA0320FFF76DFD041ECAD100F097
:103900006BFA80230322DB053C605A629C6200F064
:10391000DBF9039B002B01D1FFF776FD0298FEF740
:103920005FF8B8E700C0004090C8004000C8004001
:103930000100000694C8004007B50002019104226E
:10394000000A01A9FFF724FF0EBD000073B50500B2
:1039500005240B4AA3005B429B1819686B46DE1DC9
:103960003000FFF7A7FA022804D133782B55013C29
:10397000EFD276BD052CFCD00128FAD10230F8E751
:10398000140900111F2807D8012380228340D20583
:1039900091680B43936070473F2808D80123802229
:1039A00020388340D20551690B435361F3E75F2808
:1039B000F1D80123802240388340D205116A0B439D
:1039C0001362E8E71F2807D8012280218240C90539
:1039D0008B6893438B6070473F2808D80122802171
:1039E00020388240C9054B6993434B61F3E75F2858
:1039F000F1D80122802140388240C9050B6A9343E7
:103A00000B62E8E71F2810D880230200DB05153A77
:103A10001968012A06D820229143196019680A43BF
:103A20001A60704701228240F6E73F2811D88023B0
:103A30000200DB05353AD968032A06D810229143E3
:103A4000D960D9680A43DA60EBE701222038824066
:103A5000F5E75F28E5D842238022181A413B8340CE
:103A6000D205516A99435162516A0B435362D8E7B8
:103A700010B50400012813D1A022184992050B6843
:103A80005B015B0913430B60154B164A1968114023
:103A9000154A0A431A60402219680A431A6010BD89
:103AA0000028FCD101000A2000F0E6F821000B20DC
:103AB00000F0E2F8C0220A4B920019680A43402144
:103AC0001A601A688A431A60B022044912060B6809
:103AD0005B015B0913430B60E1E7C04614F0004053
:103AE0001CF000407F00FEFF80FD010072B6074A17
:103AF0001368013313600422054B1A600023054A42
:103B000013608022D2055360FEE7C0467808FF1F8D
:103B1000C0F00040C4F0004005490B68002B05D1FF
:103B2000044A0A6004490A60044A13607047C046A8
:103B3000140AFF1F841E0000380AFF1FC4F0004053
:103B40000023034A1360034A1360034A136070475B
:103B500054F0004040F1004044F1004002B471468E
:103B600049084900095649008E4402BC7047C046C6
:103B700002B4714649084900095C49008E4402BC00
:103B80007047C04603B47146490840004900095ACD
:103B900049008E4403BC704701B40248844601BC0E
:103BA000604700BFED6B010001B40248844601BCD0
:103BB000604700BFE927000001B40248844601BC09
:103BC000604700BF21A9000001B40248844601BC3F
:103BD000604700BF496D010001B40248844601BC42
:103BE000604700BF156B010001B40248844601BC68
:103BF000604700BF016C010001B40248844601BC6B
:103C0000604700BF2D6C010001B40248844601BC2E
:103C1000604700BFF935010001B40248844601BC89
:103C2000604700BF7997000001B40248844601BC98
:103C3000604700BFF90D010001B40248844601BC91
:103C4000604700BF2144000001B40248844601BC23
:103C5000604700BFB70E000001B40248844601BCB3
:103C6000604700BFC95C010001B40248844601BC42
:103C7000604700BFED68010001B40248844601BC02
:103C8000604700BFB5A3001101B40248844601BCDF
:103C9000604700BFCD4C010001B40248844601BC1E
:103CA000604700BFBD0B010001B40248844601BC5F
:103CB000604700BFE917010001B40248844601BC17
:103CC000604700BF8D11010001B40248844601BC69
:103CD000604700BF9DA9000001B40248844601BCB2
:103CE000604700BF6137010001B40248844601BC4F
:103CF000604700BFD9B0000001B40248844601BC4F
:103D0000604700BF116E000001B40248844601BC48
:103D1000604700BF8944000001B40248844601BCEA
:103D2000604700BF0189000001B40248844601BC1D
:103D3000604700BF8552010001B40248844601BCBF
:103D4000604700BFC1A5000001B40248844601BC21
:103D5000604700BF8B52010001B40248844601BC99
:103D6000604700BFE9D4000001B40248844601BCAA
:103D7000604700BFC56D010001B40248844601BC24
:103D8000604700BF75F8000001B40248844601BCDA
:103D9000604700BF9573010001B40248844601BC2E
:103DA000604700BF8512010001B40248844601BC8F
:103DB000604700BF7912010001B40248844601BC8B
:103DC000604700BFB352010001B40248844601BC01
:103DD000604700BF5976010001B40248844601BC27
:103DE000604700BF75A9000001B40248844601BCC9
:103DF000604700BFA9D8000001B40248844601BC56
:103E0000604700BF85C1000001B40248844601BC80
:103E1000604700BFBD5C010001B40248844601BC9C
:103E2000604700BF71B0000001B40248844601BC85
:103E3000604700BF53B9000001B40248844601BC8A
:103E4000604700BFE512010001B40248844601BC8E
:103E5000604700BFA1AF000001B40248844601BC26
:103E6000604700BFD1AE000001B40248844601BCE7
:103E7000604700BFF9ED000001B40248844601BC70
:103E8000604700BFC9A9000001B40248844601BCD4
:103E9000604700BF6D0B010001B40248844601BCBD
:103EA000604700BFE9F6000001B40248844601BC47
:103EB000604700BF01D7000001B40248844601BC3E
:103EC000604700BFDD3F000001B40248844601BCEA
:103ED000604700BF0D52010001B40248844601BC96
:103EE000604700BFDD0A010001B40248844601BCFE
:103EF000604700BF5DB7001101B40248844601BCB1
:103F0000604700BF8D82000001B40248844601BCB6
:103F1000604700BF9D6A000001B40248844601BCAE
:103F2000604700BF0134010001B40248844601BC6F
:103F3000604700BFE90B010001B40248844601BCA0
:103F4000604700BF19FA000001B40248844601BC72
:103F5000604700BF6911010001B40248844601BCFA
:103F6000604700BF6DF6000001B40248844601BC02
:103F7000604700BFC166010001B40248844601BC2D
:103F8000604700BF090E000001B40248844601BC2E
:103F9000604700BF51B8000001B40248844601BC2C
:103FA000604700BFF535010001B40248844601BCFA
:103FB000604700BFDD0C010001B40248844601BC2B
:103FC000604700BF3D71010001B40248844601BC56
:103FD000604700BFC1F7000001B40248844601BC3D
:103FE000604700BF0167010001B40248844601BC7C
:103FF000604700BFE94C010001B40248844601BC9F
:10400000604700BFADAE000001B40248844601BC69
:10401000604700BF0534010001B40248844601BC7A
:10402000604700BFC115010001B40248844601BCCD
:10403000604700BF8914010001B40248844601BCF6
:10404000604700BFEDA5000001B40248844601BCF2
:10405000604700BFCD0C010001B40248844601BC9A
:10406000604700BF8937010001B40248844601BCA3
:10407000604700BFD544010001B40248844601BC3A
:10408000604700BF0934010001B40248844601BC06
:10409000604700BF4DF9000001B40248844601BCEE
:0840A000604700BF090E00009B
:1040A800020000002EC000110100000020BE001117
:1040B800020000002AC0001101000000E840FF1FB4
:1040C8000200000028BE0011010000002862FF1F46
:1040D8000200000028C00011030000009C61FF1FBF
:1040E80012000000020000002EC0001101000000B4
:1040F80068BE0011020000002AC000110100000083
:1041080065BE00110200000072BE0011030000002D
:10411800D761FF1F0200000028C000110300000043
:10412800EC61FF1F020000002AC00011010000001E
:1041380064BE00110200000070BE00110300000000
:10414800AD61FF1F0200000028C00011030000003D
:10415800CE61FF1F020000002EC000110100000008
:10416800ACBE0011020000002AC0001101000000CE
:104178003142FF1F02000000BEBE00110100000016
:10418800A3BE0011020000002AC0001101000000B7
:104198003042FF1F02000000BCBE001101000000F9
:1041A800F461FF1F020000002AC000110100000096
:1041B8002F42FF1F02000000BABE001101000000DC
:1041C80093BE0011020000002AC000110100000087
:1041D8002E42FF1F02000000B8BE001101000000BF
:1041E8008EBE0011020000002AC00011010000006C
:1041F8002D42FF1F02000000B6BE001101000000A2
:1042080089BE0011020000002AC000110100000050
:104218002C42FF1F02000000B4BE00110100000084
:1042280084BE001102020202020200000000000027
:1042380016150000CD4C0011934C00111CBF001145
:1042480090011D0018001800FFFF07010203040574
:104258000602010600000000000000000000000047
:104268000000000000000000000000000000000046
:1042780003000000020000002EC000110100000031
:104288003CBF0011020000002AC00011010000001C
:10429800EC42FF1F0200000046BF001101000000B1
:1042A8002262FF1F0200000028C000110300000066
:1042B8008C64FF1F020000002AC0001101000000EA
:1042C800EC42FF1F0200000044BF00110100000083
:1042D8002462FF1F0200000028C000110300000034
:1042E8008464FF1F120800000000000000C6C6001A
:1042F8000000000000000000131100000001000091
:1043080000000111FFFF000050485936000000006E
:10431800000000000B000500F0000000B4000028B9
:10432800002800283075A000A000A000A000000808
:104338000008E001F000100010001000100010004C
:10434800100050005000500010001000D00700006E
:10435800000000000F000100050030750700100084
:10436800010081FF00000000FF0000009D750011A2
:10437800A573001135710011FFFF0100FF00000057
:10438800B99F0011359D00114D9C001100000000DF
:104398000000000000000800040000003B000108C5
:1043A8005902E00188212800FF00000002000000F7
:1043B8002EC0001101000000F4C00011020000002E
:1043C8002AC00011010000003144FF1F0200000054
:1043D80026C00011010000005068FF1F0200000005
:1043E8002AC00011010000003044FF1F0200000035
:1043F80024C00011010000002E44FF1F020000002D
:104408002AC00011010000002C44FF1F0200000018
:1044180022C00011010000002444FF1F18001800EA
:104428001D009001020000030202000002000000CB
:104438002EC000110100000008C100110200000098
:104448002AC00011010000007444FF1F0200000090
:1044580020C0001100000000000000000200000061
:0E44680028C00011030000007068FF1F20FF35
:040000051FFF184180
:00000001FF
